:020000040800F2
:1000000000800120210300089D480008994800084D
:100010009B48000891300008FF5D000800000000C8
:10002000000000000000000000000000AF480008D1
:100030009330000800000000AD480008754A000831
:100040003B0300083B0300083B0300083B03000898
:100050003B0300083B0300083B0300083B03000888
:100060003B0300083B0300083B0300083B03000878
:100070003B0300083B0300083B0300083B03000868
:100080003B0300083B0300083B030008000000009E
:100090000000000000000000000000003B0300081A
:1000A0003B0300083B0300083B0300083B03000838
:1000B0003B0300083B0300083B0300083B03000828
:1000C0003B0300083B0300083B0300083B03000818
:1000D0003B0300083B0300083B030008000000004E
:1000E0003B0300083B0300083B030008000000003E
:1000F0000000000000000000000000003B030008BA
:10010000000000003B0300083B0300083B0300081D
:1001100000000000000000000000000000000000DF
:100120003B0300083B0300083B0300083B030008B7
:100130003B03000800000000000000000000000079
:10014000000000000000000000000000A1480008BE
:100150003B0300083B0300083B0300083B03000887
:100160003B0300083B030008000000000000000003
:10017000000000000000000000000000000000007F
:10018000000000003B030008000000000000000029
:100190003B03000800F002F800F0B8F80AA090E86D
:1001A000000C82448344AAF10107DA4501D100F032
:1001B000ADF8AFF2090EBAE80F0013F0010F18BF47
:1001C000FB1A43F001031847C8BD0000E8BD00005A
:1001D0000A444FF0000C10F8013B13F0070408BF6D
:1001E00010F8014B1D1108BF10F8015B641E05D00B
:1001F00010F8016B641E01F8016BF9D113F0080FC0
:100200001EBF10F8014BAD1C0C1B09D16D1E58BF51
:1002100001F801CBFAD505E014F8016B01F8016B88
:100220006D1EF9D59142D6D37047000000230024FB
:1002300000250026103A28BF78C1FBD8520728BFF6
:1002400030C148BF0B6070476E2900F07686702978
:1002500000F0858166290AF0178465290AF0148464
:1002600067290AF0118461290AF0108403681B0AC7
:1002700028BF41F08001692900F0F680642900F070
:10028000F380752900F0F0806F2900F04787782906
:1002900000F05181E92900F0E186E42900F0DE86D2
:1002A000F52900F0DB86EF2900F04487F82900F0FB
:1002B00050810368DB0928BF41F08001632901F008
:1002C0006987732901F06E87E32901F07987F329A3
:1002D00001F07E87002070471FB50AF0D0FB9DE833
:1002E000030000F039FD02F0F1F9040000200021C4
:1002F0000AF074FB401C6060002000210AF058FBEB
:10030000E06001F085FA00F0F5FC1FBD09F01CF873
:100310001146FFF7E1FF02F0AEFE09F045FA0000DA
:100320000648804706480047FEE7FEE7FEE7FEE78F
:10033000FEE7FEE7FEE7FEE7FEE7FEE7094B000803
:100340009501000870B5064600F0E6FC056806F168
:100350000B0020F00704B4429CBF002070BD2B4668
:100360006A68BAB11068A04210D304F1080188424B
:100370003CBF5068586007D351681019416011683C
:10038000091B016058601460101D70BD134652684F
:10039000002AE7D12146284600F0CAFC0028DED119
:1003A00070BD70B50446051F00F0B6FC0068002C57
:1003B00014BF446870BD002C18BFAC423CBF20463F
:1003C0006468F8D301680A18AA4218BF456003D1CF
:1003D0002A6805461144016028684119A1421CBFE2
:1003E0006C6070BD6168696021680844286070BDF8
:1003F000B2F120030AD5C2F1200301FA02F120FA7A
:1004000003F300FA02F041EA0301704700FA03F136
:100410004FF00000704700001CB50C46064B7B44B3
:1004200069460090204600F0A2FD0446002069467F
:1004300000F0B0FD20461CBD730B00000FB41CB5CE
:10044000084B06AA7B4469460090059800F08FFD92
:1004500004460020694600F09DFD20461CBC5DF866
:1004600014FB00004D0B00002DE9F041064600246E
:1004700010687529314616A510D000F0CAFC002876
:1004800002DA404213A507E031688A0701D512A5B8
:1004900002E0490704D511A5012401E000F0C2FCE7
:1004A00000210A2206F1240709E0B0FBF2FCB0FBB0
:1004B000F2F302FB1C00303078541846491C002827
:1004C000F3D123462A463046BDE8F04100F0DCBCBB
:1004D000000000002D0000002B00000020000000A4
:1004E000F0B40D460188090502D5214C7C4402E098
:1004F0001F4C7C440E34002100F1240608E002F079
:100500000F071209E75D42EA03721B097754491C81
:1005100052EA0307F3D102780023120704D5702DA5
:1005200006D009B1022311342246F0BC00F0ACBC65
:1005300001231034F8E770B504460D4621461068D3
:1005400000F070FC024629462046BDE870400023BA
:10055000C6E7D21D22F00703D3E90023C0E70368F2
:10056000126843F0200303600823C3610023B7E748
:1005700054B700002DE9F05F894604464FF0000AA9
:10058000DFF874B1FB44C0F820A02046E16888473A
:10059000002874D0252806D0D4E901219047206A8C
:1005A000401C2062F1E700265F462046E16888474C
:1005B0002028054607DB312D05D2781910F8200CCC
:1005C00008B10643F1E7B00701D526F00406C4F8E8
:1005D0001CA00027C4F818A02A2D09D0284608F02E
:1005E000BBFE38B304EB8708303DC8F8185019E05B
:1005F00059F8041B204604EB87029161E1688847A3
:10060000012F054618D1E069002820DA26F02006DF
:100610001DE0D8F8180000EB800005EB40003038F2
:10062000C8F818002046E1688847054608F094FE9F
:100630000028EED1012F0AD02E2D08D12046E168E6
:1006400088477F1C0546022F46F02006C4DBA069C0
:10065000002803DA404246F00106A061F00701D00D
:1006600026F010066C2D0BD0682D09D04C2D39D0FA
:100670006A2D35D0742D35D07A2D33D016E038E080
:10068000E1682F4620468847B842054609D16C2FBD
:1006900026D04FF48060E16806432046884705462F
:1006A00004E06C2F1AD04FF4807006430DB3A5F10F
:1006B0004100192802D8203546F400664A462946EA
:1006C000204626604E46FFF7BFFD80B101280BD0C3
:1006D000F61D26F0070000F1080956E74020E4E780
:1006E0008020D8E70020D6E706F104094DE7284628
:1006F00052E7206ABDE8F09FE4B600000FB400B5F1
:100700008DB010A9099000910B904FF0FF300A9026
:1007100000200C90064878440690064878446A46C3
:1007200007900F9909A800F023FD0DB05DF814FBA8
:10073000770A00008F0A00002DE9FF5F1D464FF089
:10074000FF3B91464FF000085F46D5E90146A96995
:1007500001987F1C8847296A824688470028F6D17D
:10076000BAF1FF3F0CD0002E24F4C06419DD6006FE
:1007700014D5BAF12B0F09D0BAF12D0F0ED103E029
:10078000584604B0BDE8F09F44F48064A96901981C
:100790007F1C8847761E8246002E02DDBAF1300F9C
:1007A00003D0B9F1000F26D032E0A969761E019876
:1007B0007F1C44F400748847002E824605DDBAF1A0
:1007C000780F06D0BAF1580F03D0B9F1000F10D04E
:1007D0001EE0B9F1000F02D0B9F1100F18D1A969CC
:1007E000761E01987F1C24F40074884782461020EE
:1007F00002E0082000E00A20814609E0A96908FB20
:100800000908761E01987F1C44F4007488478246CC
:10081000002E05DD4946504600F096FC0028EDDA32
:10082000E96901988847A00502D46FF00100A8E7A4
:10083000E00725D1600613D5600502D5C8F1000098
:1008400000E0404629680A1D2A600968220501D592
:10085000087015E0220701D5088011E008600FE05C
:100860002868011D29600068210502D580F80080F4
:1008700006E0210702D5A0F8008001E0C0F8008062
:1008800038467EE770B50446C068810713D08006FD
:1008900001D5A56A04E0A169606808442169451A88
:1008A000204600F071FF002206462946204600F04F
:1008B00097FE304670BD002070BD70B510B1BDE828
:1008C0007040DFE70025074C6E1E07E02046FFF76B
:1008D000D9FF00B13546206D20F00104002CF5D180
:1008E000284670BDEC2900202DE9F0410C46074652
:1008F0001646104600F078F82078611C61280AD06E
:10090000722802D077283CD102E00125002405E0BE
:100910000225042402E0082448F2020511F8010B24
:100920002B2806D0622809D011F8010C74280AD0AF
:100930000BE045F0030544F00204EFE745F0040541
:1009400044F00104EAE744F010043846214608F078
:1009500049FD411C15D00021316171604FF40071D7
:10096000F560F1617061200704D530460222002154
:1009700000F036FE306D40F0010030653046BDE8D5
:10098000F0810020FBE72DE9F0410D460646104CB2
:10099000206DC10704D0410804D020F00104F7E71E
:1009A00022460EE05420FFF7CDFC07000ED0206D4C
:1009B00047F00101084354212065384600F032F920
:1009C0003A4629463046BDE8F0418DE70020D6E79B
:1009D000EC29002011B14FF4807201E04FF48062E5
:1009E0004FF4007300F078BE2DE9F04704464FF055
:1009F00000094FF0FF37C568D4E90486A80707D07F
:100A0000204600F0C1FE304608F0AEFC002802DAB5
:100A10003846BDE8F087280502D54046FFF7C1FCFF
:100A20004C21204600F0FEF8206D20F001002065EA
:100A30004846EEE72DE9F041074615460E461020E0
:100A4000FFF780FC04000AD06760C4E9026500F08B
:100A500067F90168216004600020BDE8F081012091
:100A6000FBE710B5431C02E010F8011B71B18107D0
:100A7000FAD14FF0013202C88C1A8C4314EAC21129
:100A8000F9D0C01A0A0603D0C01E10BDC01A10BD8E
:100A90000A0401D0801E10BD0902FCD0401E10BD0A
:100AA00040EA010370B59B072ED14FF00136042AAE
:100AB0002AD308C810C99D1B9D43121F15EAC615ED
:100AC00017D0D8B2E1B2401A50EA056110D198B2FD
:100AD000A1B2401A50EA05410AD123F07F4024F028
:100AE0007F41401A50EA052102D1180EA0EB146094
:100AF00070BDA342DBD018BA21BA884201D90120C7
:100B000070BD4FF0FF3070BD0AB9002070BD10F805
:100B1000013B11F8014B63B1A3420AD1521E08D028
:100B200010F8013B11F8014B1BB1A34201D1521E39
:100B3000EDD1181B70BD032A40F2308010F0030C79
:100B400000F0158011F8013BBCF1020F624498BF20
:100B500011F801CB00F8013B38BF11F8013BA2F1BD
:100B6000040298BF00F801CB38BF00F8013B11F038
:100B7000030300F02580083AC0F0088051F8043BD8
:100B8000083A51F804CBA0E80810F5E7121D5CBF45
:100B900051F8043B40F8043BAFF30080D20724BF78
:100BA00011F8013B11F801CB48BF11F8012B24BF0C
:100BB00000F8013B00F801CB48BF00F8012B70475B
:100BC00010B5203AC0F00B80B1E81850203AA0E8E8
:100BD0001850B1E81850A0E81850BFF4F5AF5FEA1C
:100BE000027C24BFB1E81850A0E8185044BF18C9CF
:100BF00018C0BDE810405FEA827C24BF51F8043B76
:100C000040F8043B08BF7047D20728BF31F8023BC9
:100C100048BF11F8012B28BF20F8023B48BF00F85D
:100C2000012B70474FF0000200B5134694469646DC
:100C3000203922BFA0E80C50A0E80C50B1F12001EF
:100C4000BFF4F7AF090728BFA0E80C5048BF0CC09D
:100C50005DF804EB890028BF40F8042B08BF7047FB
:100C600048BF20F8022B11F0804F18BF00F8012B6D
:100C7000704700004FF0013C50F8042B51F8043B42
:100C80009A4221D1A2EB0C03934313EACC1317D160
:100C900050F8042B51F8043B9A4215D1A2EB0C03F7
:100CA000934313EACC130BD150F8042B51F8043BB7
:100CB0009A4209D1A2EB0C03934313EACC13DBD085
:100CC0004FF00000704700BFD01A01BAB1FA81F1AD
:100CD00001F0180122FA01F0CB40C1F12001DBB292
:100CE000C0B2C01A2CFA01F3D11A914311EAC31110
:100CF000E6D1704770B5064C7C44064D7D4403E058
:100D0000206820448047241DAC42F9D170BD00000A
:100D1000E0B30000E4B3000000487047E82A002078
:100D200000487047EC2A00207047704770477047B2
:100D300038B504460A460020694601F09CFC0028AC
:100D400008BF38BD02460099204600F025FE01206C
:100D500038BD012001F064BCF8B501F081FC054606
:100D600000200C46102000BF0646A819A0420DD94D
:100D700032466946002001F07EFC070008BF01F002
:100D80004FFC0098A04218BF0546C419FFF7C4FFE6
:100D900005600746F01D20F007004619284600F0C0
:100DA0000AF8B44208BFF8BDA21B31463868BDE856
:100DB000F84000F0F1BD00210160C0E9011070476A
:100DC0001020704770B5044685690068C10601D5DA
:100DD000302600E02026C00707D070BDD4E90121ED
:100DE00030469047206A401C20626D1EF6D570BDCB
:100DF00070B5044685690078C00707D170BDD4E995
:100E0000012120209047206A401C20626D1EF6D5EB
:100E100070BD09684A0501D540B27047C905FCD5C7
:100E200000B2704709684A0501D5C0B27047C905CC
:100E3000FCD580B2704770B50C460546012A05D036
:100E40002878800600D5EA69002302E0012305E046
:100E50005B1C934202D2E05C0028F9D1A869E61835
:100E6000C01AA861286A184428622846FFF7AAFF1A
:100E700004E0D5E9012114F8010B9047B442F8D3FE
:100E80002846FFF7B5FF70BD2DE9F0470D4699469E
:100E90009246044600F124080168880604D5E069FA
:100EA00021F01001216000E00120A84201DD471B74
:100EB00000E00027A1697A1902EB0900081AA06175
:100EC0002078C00602D42046FFF77CFF002608E009
:100ED000D4E901211AF806009047206A401C761CCC
:100EE00020624E45F4DB2078C0060AD52046FFF785
:100EF00069FF06E0D4E9012130209047206A401CB8
:100F00002062381EA7F10107F4DC07E0D4E90121D3
:100F100018F805009047206A401C2062281EA5F1A1
:100F20000105F3DC2046FFF763FF2078000602D5B9
:100F30000220BDE8F0870120FBE711680268006A23
:100F4000530501D508700AE0D30501D5088006E0F5
:100F5000130603D5C217C1E9000200E008600120B2
:100F60007047000001694A1C02610878704700B5AB
:100F70008FB0CDE901310021059105497944CDE9D2
:100F8000031011466846FFF7F5FA0FB000BD0000E8
:100F9000E5FFFFFF0A6802F8010B0A6070470000D6
:100FA0002DE9FF5F15468A460446DFF8AC80F84419
:100FB0000027D8E900103E46CDE9001010E03AF8CD
:100FC00016106A4602A801F0FFFA411C07D02178EA
:100FD000890603D5E269391891420DD80744761C79
:100FE0002078800602D5E069B84205DDAE42E6DB36
:100FF0003AF816000028E2D1A069C01BA061204683
:10100000FFF7E0FED8E90010CDE90010002017E05E
:101010003AF818106A4602A801F0D6FAB0F1FF3F7C
:1010200081460BD000250DF1080B05E0D4E9012124
:101030001BF8050090476D1C4D45F7D308F10100E2
:10104000B0428046E4DB206A384420622046FFF745
:10105000CFFEBDE8FF9F0000CEAC00002DE9F041BF
:101060008046D21D22F007020025D2E90002F529B0
:1010700015A614D0011E72F1000106DA0023D0EB90
:10108000030063EB020211A608E0D8F800108B07FA
:1010900001D50FA602E0490701D50EA6012511468C
:1010A000002408F1240704E000F090FC30323A55A7
:1010B000641C50EA0102F7D12B46324621464046D5
:1010C000BDE8F041FFF7E0BE000000002D00000089
:1010D0002B0000002000000030B4002100F12404A7
:1010E00008E002F00705D208303542EA4372DB0817
:1010F0006554491C52EA0305F3D10468002310A289
:10110000250708D504F020040C4304D0C46901234A
:101110000CA2641EC46130BCFFF7B6BE10B5044615
:1011200021461068FFF77EFE02462046BDE81040CB
:101130000023D1E7D21D22F00701D1E90023CBE73C
:1011400000000000300000003A2800D2303820F0C3
:101150002002412A01D3A2F13700884201D34FF087
:10116000FF307047026811441378016018467047D9
:10117000D1600549794451610449794411620021E3
:101180001161114601F028B8EDFFFFFFD9080000FA
:10119000426842B1016811F8013B23B1521EC0E917
:1011A0000012184670470121C160881E70474268CE
:1011B0005AB1C368016843B983688B4205D0491EA0
:1011C000521CC0E90012002070474FF0FF307047FA
:1011D00070B50D4601461446D36850692A4608F09A
:1011E000DDF9002807DA411C07D0E16820F0004053
:1011F00041F48041E160281A70BD204600F090FA69
:101200004FF0FF3070BDC1680022026021F48051B0
:1012100041F0400111F4C06FC16001D0826070479D
:1012200002694168891AC269891A816070472DE98B
:10123000F0470446C06840F48000E060010312D526
:1012400020F40020E060810606D4E26A61688A42E8
:1012500000D80A46511A216040F40010E06094F86A
:101260002500BDE8F08720F40010E060800602D57C
:10127000204600F0ACFAE06842F281014FF0FF39FD
:101280000140012903D0204600F04AFAB6E0216867
:10129000002600290ADAC94340F480502160C4E9DD
:1012A00002606068411C61600078DAE744F2400146
:1012B00008420CD020F4A04040F040002660E060DE
:1012C00021696068401AE169401AA06096E02169CE
:1012D00091B9C00310D4E069FFF734F82061B0B1D0
:1012E000E06840F4006010F4407FE06002D140F418
:1012F0008070E06020696060E068D4F814A0C106E6
:101300001AD5C0030ED5204600F03EFA14E004F1D1
:10131000240020610120E061E06820F4407040F486
:101320008060E6E721696068401AA169014450467F
:1013300008F05EF90028A6DBE068C0032AD56168E2
:10134000E06A884200D808462169451AE069471BCF
:101350001BD02046D4F8188000F016FA08EB0501DF
:101360005046C4F8188008F043F900288BDBE06889
:1013700040F40030E060000202D5A0692844A0617A
:10138000E1692069C91B45180DE0204600F0FCF911
:10139000E769F5E725696168D4E90607491BE56255
:1013A00008446560A061E06820F0100010F4C06F90
:1013B000E06002D0204601F0EBF8E06840F4805095
:1013C000C4E90260000205D52069E06260606FF048
:1013D000010046E7224639462846FFF7F9FE411C40
:1013E0000CD02918E16258B1401E2060681C606072
:1013F000E06840F40030E060287832E7484630E7A3
:1014000065602046FFF7FFFEF8E72DE9F047054647
:101410000C46C86820F4201040F48000C8608006A4
:1014200002D5084600F0D3F9E06841F282014FF09E
:10143000FF390140022903D0204600F071F9B5E0E0
:1014400000F42041B1F5004F0FD1C00306D561680B
:10145000E06A884200D80846606006E02069E062E1
:101460006060606907F096FFA061A0680022EEB29C
:1014700000280DDAE1688B050AD4C043A06041F46E
:1014800090302260E0606068411C61600670A5E0F9
:10149000E0689046226040F40050E060206968BB3C
:1014A000606907F08BFF012704F12405A0B1A08932
:1014B00010F4407F08D0E069FEF744FF206118B1C6
:1014C000E06840F4006016E0E7612561E06820F420
:1014D000407040F480600EE0E069FEF733FF0028C2
:1014E0002061F1D0E06840F4006010F4407FE060DB
:1014F00002D140F48070E06020696060E068256996
:101500006FF0010AC1051FD56168E06A884200D802
:101510000846411B04D02246284600F00BF9F0BBD8
:10152000E068010203D5E562C4E9015854E0691C92
:10153000E1626160E16940F48030491EC4E9021053
:1015400030462E70BDE8F087010202D500F48032EB
:101550000AE06068411C61600670E0680A2E40F491
:101560008030E06006D00022E16A6068814203D9E1
:101570000B4602E00122F7E70346A7895B1B7F05C4
:1015800003D4E7699F4200DDE2B1814200D8014601
:10159000E5620F1AC4E90158002B09DD00E005E0FF
:1015A00022461946284600F0C5F808B14846C9E762
:1015B00047B1A069E5626560C01BA061E06840F0CA
:1015C0001000E060E068000208D56168A069E5628B
:1015D000491B08446560A0615046B3E73046B1E757
:1015E0002DE9F041044616460D464769007B800709
:1015F0002ED0384607F0E2FE50BB3EB3012E02D09B
:10160000022E25D104E0204600F0A0FF05441DE095
:10161000384607F0BFFEE168002841F01001E160A4
:1016200005DA204600F07CF80120BDE8F081C9030E
:101630000BD56268E16A914200D81146A269114453
:101640002269891A814200DD08460544002D01DA2D
:101650000220EAE7E16A6068E268814206D291030B
:10166000E06203D522F4003141F01002A6690027A0
:10167000AE4213DCE16A814201D90B4600E0034629
:1016800003EB060C2369ACEB030CAC4506DD814291
:1016900001D98C4600E084469C4505D1A7602760AF
:1016A00042F02000A5620DE0AD1BE669AE1B814251
:1016B000A66000D90846C01A281A20605819606030
:1016C00022F0200003490840E060002084F84870C0
:1016D000ABE70000BFCFD7FF70B5C468A50713D034
:1016E000650211D4B2F5807F09D0B2F5007F06D033
:1016F000B2F5806F08D1012300F1240106E05D1EE0
:101700006FF07F46B54201D3012070BD0161C36116
:10171000416024F470611143C160002070BD00007D
:10172000C16821F4001141F08001C1600021816095
:10173000016070472DE9F047814614460E464FF090
:10174000FF383248D5685769054209D03846A16943
:1017500007F04EFF002811DB2C48C0430540E56030
:101760002B4632464946384607F056FFA16920F01D
:101770000042B21A11440028A16103D02046FFF7AD
:10178000CFFF4046BDE8F08770B504460569C06AE2
:101790006168884200D80846E16821F42011E160C0
:1017A000C90312D5A84208D02246411B2846FFF79C
:1017B000C1FF10B14FF0FF3070BD0020E562C4E9F9
:1017C0000150E06820F48030E060002070BD10B56A
:1017D0000446C06820F02000E060A16AA069884249
:1017E0000DD02046FFF7D0FFE06820F4405040F0D5
:1017F0001000E060A06AA0612069E062606044F2CD
:101800004001E0688843E06010BD00001000020065
:1018100010B542485421FFF705FA41485421FFF71B
:1018200001FA40485421FFF7FDF93F493B483C4A43
:101830003F4B08603D490A603A491960531C0365F3
:10184000481C1065012008653B48344A39A178449A
:10185000FFF74AF820B9384878440A3800F0D9FE32
:1018600037482F4A35A17844FFF73EF820B934486D
:1018700078440A3800F0CDFE32482A4A2FA1784435
:10188000FFF732F820B92F4878440A3800F0C1FE3B
:1018900040232248DC0000212246FFF71DFF20B133
:1018A00025487844543800F0B4FE1D4822464023B1
:1018B0000021FFF711FF20B121487844543800F08F
:1018C000A8FE1848224610230021FFF705FF002834
:1018D00006D01C487844BDE81040563800F099BE48
:1018E00010BD104870B5006D20F001040B48FFF7E3
:1018F0007BF80B48FFF778F80A48FFF775F809E01E
:10190000206D20F001052046FFF76EF82046FEF717
:1019100048FD2C46002CF3D170BD0000EC290020BE
:10192000402A0020942A0020B8020020BC02002097
:10193000C0020020720000006294000077000000E6
:1019400051940000419400002DE9F0410646FFF754
:10195000E7F98046454613E016B1E068B0420ED183
:1019600020682860D4E90101D8F800708847204633
:10197000FEF717FDD8F80000B842EBD100E025468D
:101980002C68002CE8D1BDE8F08110B500F050FEC5
:10199000BDE8104000F038BE034640688C46002881
:1019A00018BF88423CBF03464068F8D31868184403
:1019B000884207D00CF1030020F00700001D411AF7
:1019C000521A0146081D0A60FEF7EBBC30B5B0F1B3
:1019D0000A024FEA900E71F100034EEA817EB0EBED
:1019E0000E0061EB91014FEA101E4EEA017E10EBF2
:1019F0000E0041EB11114FEA102E4EEA016E10EB72
:101A00000E0041EB11214FEA104E4EEA014E10EB51
:101A10000E0041EB1141401841F100014FEAD000A6
:101A200040EA41704FEAD10110EB80054FEA810492
:101A300044EA907444EB01046D1944EB0404521B16
:101A4000A3414FF0000348BF0A3200D530BD401C0F
:101A500041F1000130BD10B5044600F02FFE0068D2
:101A6000005D00F0010010BD70472DE9FF4F0C46EE
:101A70001E464FF0FF378BB0D2E90001DDF86080E1
:101A80000A908A46C1F30A5505B93D460021084629
:101A90004FF00000BAF1000F00F4400005DA00EB4F
:101AA00080004FF4400101EA50004FEA9059B9F12B
:101AB000010F00DDB9460A9850EA4A000ED044F6FC
:101AC0001050A5F2FF3545432F14B8F1000F1ED07A
:101AD0007542291E1EDDC9F100021CE0B8F1010F9C
:101AE0004FF0000001D0302103E0F24305E0215423
:101AF000401CB042FBDB30460022002121540B99F0
:101B0000C1F80880C1E900200FB0BDE8F08FBD1B0F
:101B10006D1CDEE74A4600DA694206A800F01EFEA8
:101B200006AB93E8070003AB83E8070050460A9929
:101B300000F0E6FE8DE80700A0F500501F38009089
:101B40000398002D09DD42F21F014A46084403A90B
:101B50000390684601F045F908E0A0F500504A46B8
:101B60001F3803A90390684601F04FF98DE807007C
:101B70000004000C03D04FF0FF30410800E0104695
:101B8000B8F1000F03D00022009215461EE0751E2A
:101B900005D4FFF71BFF303262556D1EF9D5B346F1
:101BA0000122084302D000227F1C04E02078302864
:101BB00001D100227F1E002A099786D01DE0112D39
:101BC00007DAFFF703FF303262556D1C50EA01025D
:101BD000F5D1084302D00098C8B10EE00021681E7C
:101BE00005E0235C625C63542254401E491C814220
:101BF000F7DBAB46A81B401E0990002004F80B0041
:101C00000B98099AC0F80880C0E9002B7CE71126E0
:101C10004FF0000859E72DE9F04F88460446D21DE1
:101C200022F0070191B0D1E90001CDE90A0107F0E6
:101C300001FB02460B98C00F01D02D2007E0206861
:101C4000810701D52B2002E0202101EAC000032AF0
:101C5000099001D0072A05DB03464146204600F0E3
:101C60003DFD0BE12078800601D5E06900E006200B
:101C7000B8F1650F814606D0B8F1660F18D0B8F1FB
:101C8000670F70D131E00020B9F1110F009001DB36
:101C9000112301E009F101030AAA01A90CA8FFF729
:101CA000E4FEDDE90C70002609F10105834647E0FA
:101CB00001204B4600904FF000470AAA01A90CA84A
:101CC000FFF7D3FEDDE90DB00C995D46002610B993
:101CD00009F101000D18B9EB050003D4C0F1FF367E
:101CE00009F10105A5EB09002BE0B9F1010F01DABB
:101CF0004FF001090020B9F1110F0090484601DDB5
:101D0000112300E003460AAA01A90CA8FFF7ADFEC3
:101D1000DDE90C704D4600268346207800070AD482
:101D2000AB4500DA5D4601A8012D04DD411911F82B
:101D3000011C302907D04F4502DA17F1040F04DAED
:101D4000012082460FE06D1EEEE7002F02DCED1B46
:101D50003E4403E0781CA84200DD7D1CB81B00F166
:101D6000010A4FF000472078000703D4AA4501DBA1
:101D70004FF0FF3A0021B7F1004F0DF143088DF805
:101D8000431024D002202B23002F01DA7F422D2381
:101D90000A21021EA0F1010000DC5FB197FBF1FCFB
:101DA00097FBF1F201FB1C7C17460CF1300C08F894
:101DB00001CDEEE7A8F1010003702188090501D5E6
:101DC000452100E06521A0F1010800F8011C0998F7
:101DD0000FA9A1EB0807FF1D00B10120411901EB7C
:101DE000EA70A1693844081A401EA0612078C00634
:101DF00002D42046FEF7E6FF099828B1D4E9012174
:101E00009047206A401C20622078C00622D52046D8
:101E1000FEF7D8FF1EE0002E04DBB34502DD01A86B
:101E2000805D00E03020D4E901219047206A401C09
:101E30002062761CAAF101005FEA000A0AD100F0D4
:101E400045FCC0680168405CD4E901219047206AE4
:101E5000401C2062281EA5F10105DCDC07E0D4E966
:101E6000012118F8010B9047206A401C2062381E9F
:101E7000A7F10107F3DC2046FEF7BAFF032011B0FB
:101E800043E600002DE9F04F04460D46D21D22F036
:101E9000070089B0D0E900974846394607F0CAF9EB
:101EA0000246F80F01D02D2307E02068810701D5F5
:101EB0002B2302E0202101EAC0038DF820300BB172
:101EC000012000E00020032A824601D0072A04DB1B
:101ED0002946204600F002FC3FE12078800601D42C
:101EE0000D2500E0E569C7F30A560D2D49DA0021FA
:101EF0004FEA175B08464FF00000002F00F4400047
:101F000007DA00EB80004FF4400100EBD07001EAEB
:101F100060008115012901DD4FF0FF3100224FEAF9
:101F2000850CBCF1180F06D31346ACF118004FF026
:101F30008052C24003E04FF4801323FA0CF30CF1FB
:101F40000C0CBCF1200F04D3ACF1200C09FA0CF0FE
:101F500001E007FA0CF000294FF0004801DD18B944
:101F60000FE00ED140450CD319EB02095F4121B9B6
:101F7000404502D19F4329EA0209BBEB175F00D01D
:101F8000761C2088000502D57B48784402E07A4818
:101F90007844193808AA302302F80A30037C0AF181
:101FA0000101002E0AF1020A53546A4602DC4FF086
:101FB000300101E04FF031014FF001088DF80010C1
:101FC00002D0A6F2FF3603E059EA470100D06B4E7B
:101FD000002D02DC2178090704D54FF002082E21DC
:101FE0008DF80110C44600210BE0C7F303433F0105
:101FF000C35C491C6D1E02F80830052908F1010870
:1020000001DA002DF1DC00210CE000EB1973491C12
:102010001B786D1E082902F808304FEA091908F1EB
:10202000010801DA002DF0DC21688B0602D516E0EC
:10203000A8F10108E04505DD02EB080313F8013CB7
:10204000302BF5D0B8F1000F09DD02EB080313F8CF
:10205000013C2E2B03D1090701D4A8F10108002D62
:1020600005DD3E2102F808106D1E08F10108407CD4
:10207000002E02F8080008F1010804DA2D2076424B
:1020800002F8080002E02B2002F808000A214FF4B1
:102090007A70864208F101080BDB96FBF0F33033CF
:1020A00002F8083096FBF0F308F1010800FB136614
:1020B00001E0642E0CDB642096FBF0F3303302F871
:1020C000083096FBF0F308F1010800FB136601E00D
:1020D0000A2E06DB96FBF1F0303002F8080008F11A
:1020E000010896FBF1F001FB1060303002F80800A7
:1020F000A16908F1010808EB050202EB0A00081AC1
:10210000A0612078C00602D42046FEF75BFE216A5B
:1021100008AE01EB0A00206204E0D4E9012116F8C0
:10212000010B9047BAF1010AF7D22078C00602D518
:102130002046FEF747FE6E4609E016F8010B3E28E2
:102140000FD0D4E901219047206A401C2062B8F1E9
:102150000108F2D22046FEF74BFE09B00320BDE88D
:10216000F08F206A2844206203E0D4E90121302066
:1021700090476D1EEBD3F8E70D9D000002FCFFFFBA
:1021800010B5436913B1AFF3008001E0FEF753FED1
:10219000012010BD127800F124010A7000224A705B
:1021A0000122EDE711684FF0FF32E9E710B543690E
:1021B00013B1AFF3008001E0FEF7F2FE012010BD85
:1021C000128800F1240182840022C2840122EDE7FA
:1021D00011684FF0FF32E9E72DE9F34F4FF0000AA5
:1021E0000C4656468DB001200C9001F10C000B906E
:1021F00062690B9801219047051E2DD0252D2CD00A
:10220000216A8847C0B162690B9801219047216A11
:1022100088470028F7D16269411E0B98904700E07B
:10222000761CA1690D988847216A88470028F7D154
:10223000E1690D988847DBE7A1690D988847A842B6
:10224000074601D1761CD3E7E1690D9888477F1CCA
:1022500002D1BAF1000F6FD06BE162690B980027D1
:102260003D46394690472A2804D162690B980121DE
:1022700090470125DFF8D08262690B9801219047D1
:10228000A0F130010A290AD24745E5DC07EB8701B6
:1022900000EB4107303FDFD445F01005ECE7E906DD
:1022A00001D46FF000476C280AD04C2814D068285D
:1022B00015D06A280DD074281CD07A281AD01DE0B9
:1022C00062690B98012190476C2802D045F0040503
:1022D00014E045F002050DE045F020050AE06269D2
:1022E0000B9801219047682802D045F0080505E0C9
:1022F00045F4006562690B9801219047C4E90157D4
:1023000065283DD019DC58287AD00CDC452837D018
:1023100004DC252826D041289ED131E046282FD044
:10232000472899D12CE05B2877D0612828D06328F2
:102330007CD0642823D15AE0F6E06F2848D008DC2E
:1023400066281DD067281BD0692821D06E2816D199
:1023500027E0702845D0732868D0752847D07828A2
:102360000DD14DE0A1690D988847252805463FF419
:1023700069AFE1690D9888476D1C3FF46AAFD8E0FA
:102380000D9923466A466FF00100AFF30080C5E067
:1023900045F0400023464FF000026060A80736D4A5
:1023A0003EE0E8077FF447AF2068011D2160006828
:1023B000290501D506701BE7290701D5068017E717
:1023C000A90703D5F117C0E9006111E706600FE71F
:1023D00045F0400023464FF008026060A80716D47D
:1023E0001EE040F60E0125EA0100606016E045F0AF
:1023F000400023464FF00A026060A80707D40FE0B0
:1024000045F040006060A80708D5234610220D99CA
:102410006FF00100AFF3008080E007E01022234658
:102420000D996FF00100FEF787F977E04FF0000992
:1024300063284F46C8464B46CB4602D05B2806D0A1
:1024400038E0E80601D40120A060012732E062698B
:10245000D4F80CB00B98012190475E2807D14FF0BB
:10246000010949466269D4F80CB00B98904721697C
:1024700039B900210A4603AB43F82120491C082939
:10248000FADBD8B3216949B308F1010862690B98F6
:10249000012190475D28F4D1B9F1000F09D0002047
:1024A00003A951F82020D24341F82020401C0828DD
:1024B000F7DB03AB2069002820794FEA40701ED07B
:1024C0005B462246CDF80080CDE901970D990028A2
:1024D0006FF0010020DAAFF300801FE0C11703AAFC
:1024E00000EBD1614B1121F01F0102EB8302411A75
:1024F00013680120884003431360C7E719E00D9972
:10250000224600286FF00100009702DAAFF3008046
:1025100004E0AFF3008001E0AFF3008000280ADAA6
:10252000401C06D10C9820B14FF0FF300FB0BDE831
:10253000F08F5046FAE7E90701D10AF1010A064493
:1025400000200C9054E60000CCCCCC0C10B5014619
:10255000C268900703D0900607D5886A0AE000F0A9
:10256000B9F801210160881E10BD8B6948681844C4
:102570000B69C01A91F848301BB191F84910401A04
:1025800010BD1103FCD50028FADD401E10BD00006F
:1025900070B5054640F202260A4C0FE094F8500050
:1025A000C00708D0AC4206D0E06836EA000002D18D
:1025B0002046FEF767F9206D20F00104002CEDD1D4
:1025C00070BD0000EC29002070B516460C4605468B
:1025D00000F074F8036893F80101012806D0FF2C7D
:1025E0000FD8185D68B101202C7070BDD3F80701B9
:1025F0003246214603F2071303442846BDE87040E3
:1026000018474FF0FF3070BD002801D000F050B8DF
:10261000704710B500F02AF9BDE81040FFF7F4BF8D
:1026200010B500F03DF9BDE81040FFF7EDBF000028
:1026300010B5002102A000F0FFF8012010BD00003D
:102640005349475056464E3A205075726520766978
:10265000727475616C20666E2063616C6C656400D9
:10266000124B694600F580528A421A6001D8114621
:1026700070471960704730B50C4D6B46A3F5805319
:102680002C6822449A420FD89B1A02F5805003EB23
:10269000D37302EB6303984200D91846C01D20F0A3
:1026A00007020C60101B2A6030BD0000C40200202D
:1026B00001491820ABBEFEE72600020010B500F06D
:1026C00005F8001D10BD00BF1583000000487047CD
:1026D000F02A002000487047042B00202DE9F0412B
:1026E0001F46044603260168072A01F4006004DB44
:1026F00008B116A505E016A503E008B115A500E090
:1027000015A521F010002060A069C01EA0610FB1C6
:10271000401EA0612046FEF755FB4FB1D4E90121D0
:1027200038469047206A401C2062C01C206206E0A8
:10273000206AFAE7D4E9012115F8010B9047761ECB
:10274000F8D22046FEF754FBBDE8F0814E414E0022
:102750006E616E00494E4600696E66002DE9F047D5
:10276000814616468AB0334878440DC88DE80D007E
:1027700030487844801C03AC0DC884E80D0041F655
:102780009B300844372190FBF1F290FBF1F5A5F165
:10279000800501FB12041B3C02D56442012000E0CD
:1027A0000020DFF890A080460027FA44AAF1BE0A74
:1027B0000DE0E00709D03246684607EB47010AEB17
:1027C000810100F022FB8DE8070064107F1C002CC3
:1027D000EFD1184F7F44AC3F18E0E80714D007EB67
:1027E00004100DF1180A90E80E008AE80E00C06887
:1027F000F04201D198190890324606A903A800F0CA
:1028000004FB03AB83E807006D10641C002DE4D1CA
:1028100032466946B8F1000F03A802D000F0E1FA91
:1028200001E000F0F2FAC9E90001C9F808200AB095
:10283000BDE8F087C095000070B505460C460A203B
:1028400000E06D1C00F054F835B128780028F8D16C
:1028500002E0641C00F04CF814B120780028F8D194
:10286000BDE870400A2000F043B8000010B50146F2
:1028700002A0FFF7E1FF012010BD000053494752BD
:10288000545245443A2052656469726563743A2033
:1028900063616E2774206F70656E3A20000000003F
:1028A00010B5012805D0002103A0FFF7C5FF0120C6
:1028B00010BD09A1F8E7000053494752544D454D5A
:1028C0003A204F7574206F662068656170206D65D1
:1028D0006D6F7279000000003A2048656170206DCC
:1028E000656D6F727920636F7272757074656400C4
:1028F00008B569468DF800000320ABBE08BD7047DF
:102900005FEA400C08BF91F0000F4FEA8C234FEABA
:10291000C12243EA51514FEA1C5018BF00F5F04064
:102920004FEA300018BF41F000415FEA6C5C00F0F4
:102930002980BCF1FF3F08BF40F080407047130C76
:1029400006BF12044FF0100C4FF0000C130E04BF22
:1029500012020CF1080C130F04BF12010CF1040C4D
:10296000930F04BF92000CF1020CD30F04BF52006E
:102970000CF1010C11464FF00002A0F11F00A0EB7A
:102980000C00704711F0004F08BF704731F0004154
:102990003FF4D5AF0B0C06BF09044FF0100C4FF0FD
:1029A000000C0B0E04BF09020CF1080C0B0F04BF46
:1029B00009010CF1040C8B0F04BF89000CF1020C0F
:1029C000CB0F04BF49000CF1010CCCF12003A0EBAC
:1029D0000C0022FA03F302FA0CF241EA030100F1BF
:1029E0000100704720F07F4C80EA030023F07F470E
:1029F000ACEB070303F57C5300F0004003F1FF0349
:102A00002DE980494FEA154B09B44FEA144325EAF2
:102A10000B4E24EA03480FF2042606EB132749085D
:102A20003E785FEA320203FB0667C7F5000707FB43
:102A300006F64FEA54374FEAD64606F1020607FB80
:102A4000066CCCF1005C4FEA1C472CEA074C07FBF4
:102A500006F40CFB06F504EB15464FEA961634BF58
:102A600000204FF000404FEAD13706FB07FC4FEA49
:102A70001C4C0CFB0BF7D21B03FB0CF761EB0701A3
:102A80000CFB0EF7B0EB074072EB17420CFB08F79C
:102A900034BFA2EB0742B2EB074261EB17414FEAAA
:102AA0000C444FEA910706FB07FC4FEA1C4C0CFB59
:102AB0000BF7B0EBC74072EB573203FB0CF734BF98
:102AC000A2EBC742B2EBC74261EB57310CFB0EF7EA
:102AD000B0EBC70072EB57720CFB08F734BFA2EBE8
:102AE000C702B2EBC70261EB5771039F4FEA8161E6
:102AF00041EA921104EBCC044FEAD1374FEA8262EB
:102B000006FB07FC42EA90124FEA80604FEA1C4C39
:102B10000CFB0BF7D21B03FB0CF761EB07010CFB63
:102B20000EF7B0EB074072EB17420CFB08F734BF0F
:102B3000A2EB0742B2EB074261EB17414FEA8C551B
:102B40004FEA910704EB9C2406FB07FC4FEA1C4C60
:102B50000CFB0BF7B0EBC74072EB573203FB0CF7E3
:102B600034BFA2EBC742B2EBC74261EB57310CFB5B
:102B70000EF7B0EBC70072EB57720CFB08F734BFCF
:102B8000A2EBC702B2EBC70261EB577115EB4C2504
:102B90004FEA816141EA92114FEA82624FEAD137EE
:102BA00042EA901206FB07FC44F100044FEA806001
:102BB0004FEA1C4C0CFB0BF7D21B03FB0CF761EB31
:102BC00007010CFB0EF7B0EB074072EB17420CFB52
:102BD00008F734BFA2EB0742B2EB074261EB1741A3
:102BE00015EB1C154FEA813141EA92414FEA8232DE
:102BF00042EA90424FEA80304FEA0C7644F10004FA
:102C000048EA03434EEA0B484FF0000EB2EB080CC3
:102C100071EB030724BF624639464EEB0E0E4FF0B0
:102C2000000B0018524149414BEB0B0BB2EB080C67
:102C300071EB03077BF1000B24BF624639464EEB74
:102C40000E0E4FF0000B0018524149414BEB0B0B9D
:102C5000B2EB080C71EB03077BF1000B24BF62465B
:102C600039464EEB0E0E51EA020718BF46F0010638
:102C700016EB0E7655F1000254F1000103D5BDE8C4
:102C80008901BDE80088BDE88901BDE80048B619A2
:102C9000524141EB0101A3F10103704780807F7E27
:102CA0007D7C7B7A797877767675747372717170C2
:102CB0006F6E6E6D6C6C6B6A6A6968686766666574
:102CC0006464636362616160605F5F5E5E5D5D5C02
:102CD0005C5B5B5A5A595958585757565655555573
:102CE0005454535352525251515050504F4F4F4ED3
:102CF0004E4D4D4D4C4C4C4B4B4B4A4A4A49494921
:102D00004848484747474746464645454544444462
:102D1000444343434342424242414141002B26D473
:102D2000770021D01CB54FEA370703B44FF01000ED
:102D30004FF010014FF000000FBCBDE810400BF148
:102D4000010BBBF1010F08BF5FEA170722BF12F1A9
:102D5000010211F101014FF0004143F1000300F0C5
:102D6000004043EA00007047F9D35708DAE746EA23
:102D7000064613F1400F4FEA16461FDD13F1200FF0
:102D8000DFBF16430A46002120335B42C8D0C3F19F
:102D9000200746EA064602FA07F74FEA164646EAD1
:102DA0000706C3F1200722FA03F201FA07F721FA16
:102DB00003F14FF0000342EA0702B1E746EA0206D8
:102DC00046EA06464FEA164646EA0106BCBF46EA10
:102DD0000646360C4FF000034FF000024FF00001A2
:102DE0009EE72DE9C048934630B491E8380007C803
:102DF00031EA400C48BF34EA430C03D5FFF7F2FD3B
:102E0000FFF78CFFF0BCBDE800882DE9C048934671
:102E100030B491E8380007C810F0804F08BF13F0B5
:102E2000804F03D100F005F8FFF778FFF0BCBDE854
:102E3000008820F07F4780EA030023F07F4C07EBF7
:102E40000C03A3F57C5300F00040A3F1FE0392F0C5
:102E5000000F00F0B38095F0000F00F077802DE9AF
:102E600001494FEA11404FEA144621EA004800FBAD
:102E700006FC24EA064708FB06F607FB08F800FBF9
:102E800007F718EB06484CEB164C4FEA124B18EBC1
:102E900007484FEA15464CEB174022EA0B4E0BFB56
:102EA00006FC25EA06470EFB06F607FB0EFE0BFBAB
:102EB00007F71EEB064E4CEB164C4FF000061EEBD0
:102EC000074E4CEB174B18EB0B0840F1000018EBCA
:102ED0000E0B58EB000840F100008F1A4FF0000174
:102EE0003CBFC943661B14BFB5EB040C00213CBFBB
:102EF000C943F61B4FEA17444EEA8E0E27EA0445F3
:102F00004FEA1C4704FB07622CEA074C05FB07F756
:102F10000CFB05F604FB0CFC16EB074642EB1742D4
:102F200016EB0C4642EB1C421BEB060658EB02026A
:102F3000414146EA9E0601D5BDE80189B6195241D4
:102F400041EB0101A3F10103BDE801894FEA1445FA
:102F50004FEA114724EA054621EA074C05FB07F42E
:102F600006FB07F70CFB06F105FB0CFC11EB074118
:102F700044EB17444FEA124711EB0C4144EB1C445D
:102F800022EA074C05FB07F206FB07F70CFB06F6E7
:102F900005FB0CFC16EB074642EB174216EB0C4602
:102FA00042EB1C456A1854F1000148BF7047B6193E
:102FB000524141EB0101A3F10103704795F0000F6D
:102FC00037D04FEA11424FEA144721EA024624EA79
:102FD000074C02FB07F106FB07F70CFB06F402FBAC
:102FE0000CFC14EB074441EB17414FEA154714EB77
:102FF0000C4441EB1C4125EA074C02FB07F506FB9C
:1030000007F70CFB06F602FB0CFC16EB074645EB3C
:10301000174516EB0C4645EB1C42121951F1000105
:1030200048BF7047B619524141EB0101A3F10103BA
:1030300070474FEA14454FEA114724EA054621EA52
:10304000074C05FB07F106FB07F70CFB06F24FF0F8
:10305000000605FB0CFC12EB074241EB174112EB9B
:103060000C4251EB1C4148BF7047921841EB0101E3
:10307000A3F10103704710B506F087FF06F084FF47
:10308000BDE8104006F08EBE00210160C1607047AF
:10309000FEE77047002251B1012908BF4FF480724A
:1030A00005D002290CBF4FF400724FF440720E4954
:1030B0000B6823F440730B600B681A430A600A68BC
:1030C00022F0F8020A600A68F82393FAA3F3B3FA2D
:1030D00083F3984040F0020010430860086840F411
:1030E0008030086070470000103C024020490868AA
:1030F00010F0100F1F4805D0C26942F01002C261E3
:1031000010220A600A6812F0200F05D0C26942F04E
:103110000802C26120220A600A6812F0400F05D03E
:10312000C26942F00402C26140220A600A6812F0D9
:10313000800F05D0C26942F00202C26180220A609B
:103140000A6812F4807F06D0C26942F00102C261AF
:103150004FF480720A600A6812F0020F08BF7047CD
:10316000C26942F02002C26102200860704700007C
:103170000C3C0240DC07002070B5174904460020D3
:10318000C86100F0C9F9154D0646286810F4803F63
:103190000FD000BFB4F1FF3F07D024B100F0BCF95D
:1031A000801BA04201D9032070BD286810F4803F25
:1031B000F0D1286810F0010F1CBF0120286028689A
:1031C0004FF4F97131EA00001CBF002070BDFFF719
:1031D0008DFF012070BD0000DC0700200C3C024088
:1031E00090F83510022903D08021416501207047F5
:1031F000052180F835100068016821F001010160A7
:10320000002070470348016841F000410160002040
:1032100070470000103C02402DE9F0472D4F8146D9
:103220001546387E98460E46012804BF0220BDE8A8
:10323000F087012038764CF25030FFF79DFF08BB35
:10324000254CB9F1000F21D0B9F1010F2AD0206827
:10325000B9F1020F20F440702060206830D040F4B3
:1032600040702060206840F0010020603560C6F8A2
:10327000048000BF4CF25030FFF77EFF216821F040
:103280000101216000213976BDE8F087206820F433
:103290004070206020682060206840F001002060BD
:1032A0003570E7E7206820F440702060206840F423
:1032B00080702060206840F0010020603580D9E7F0
:1032C00040F400702060206840F00100206035600C
:1032D000D0E70000DC070020103C024006480068F0
:1032E00010F0004F04BF01207047044904480160FA
:1032F0000449016000207047103C024023016745EB
:10330000043C0240AB89EFCD2DE9F84F00227A4E04
:10331000DFF8E8E101274FF0030A4FF00F0800BF84
:103320000B6807FA02F42340A3427DD1D1F804C010
:10333000BCF1020F18BFBCF1120F15D14FEAD20C2D
:1033400000EB8C05D5F820904FEA427C4FEADC6C0C
:1033500008FA0CFB29EA0B09D1F810B00BFA0CFCA7
:103360004CEA090CC5F820C0D0F800904FEA420C96
:1033700091F804B00AFA0CF50BF0030B29EA0509E1
:103380000BFA0CFB4BEA0909C0F80090D1F8049045
:10339000B9F1010F18BFB9F1020F05D0B9F1110F42
:1033A00018BFB9F1120F18D1D0F80890D1F80CB0AD
:1033B00029EA05090BFA0CFB4BEA0909C0F8089049
:1033C000D0F8049029EA040491F80490C9F3001994
:1033D00009FA02F949EA04044460C468AC438D6800
:1033E00005FA0CFC4CEA040CC0F80CC0D1F804C07F
:1033F0001CF0805F79D0D6F800C04CF4804CC6F841
:1034000000C0D6F800C00CF4804CCDF800C022F00B
:10341000030C0CF1804C0CF5983CDCF80858940730
:10342000240F08FA04F900E05FE025EA0905A0F19D
:103430008049B9F5003920D0A0F18049B9F50139AA
:1034400008BF4FF0010918D0A0F18049B9F5023941
:1034500008BF4FF0020910D0A0F18049B9F5033937
:1034600008BF4FF0030908D0A0F18049B9F504392D
:103470000CBF4FF004094FF0050909FA04F42C437E
:10348000CCF80848DEF800C04C682CEA030C14F4B1
:10349000803F18BF4CEA030CCEF800C0184CD4F89B
:1034A00000C04D682CEA030C15F4003F18BF4CEA2D
:1034B000030CC4F800C0134CD4F800C04D682CEACB
:1034C000030C15F4801F18BF4CEA030CC4F800C0AD
:1034D0000D4CD4F800C04D682CEA030C15F4001F05
:1034E00018BF4CEA030CC4F800C0521C102AFFF4A9
:1034F00017AFBDE8F88F000044380240003C01409F
:10350000043C0140083C01400C3C0140002A08BF3B
:10351000090481617047000001480068704700009D
:10352000E801002002480168491C01607047000062
:10353000E80100200B4810B5016841F400710160FA
:10354000016841F480610160016841F480710160AB
:10355000032000F065F80F2000F006F800F05EF898
:10356000002010BD003C024038B52348002501680A
:1035700041F008010160006800F0080000901F4859
:10358000016841F008010160016821F00801016053
:1035900001F078FA1B4C1A481C492060681EE06054
:1035A000194800682561B0FBF1F0401EC4E901052F
:1035B0002046656100F09CFF1549322005F052FE5F
:1035C00014494FF48020C1F800010021204600F08A
:1035D000ABFF0421204600F0A7FF2068416A0E4A95
:1035E000116001F57A7181632068C16841F00401BE
:1035F000C160002038BD0000403802402038024041
:10360000000C0040C80200209801002040420F003A
:103610007DA8000804E000E094010020704700004D
:10362000074900F007000A684FF6FF031A4042EA14
:10363000002040F0FD7040F080600860704700009E
:103640000CED00E0D0F8B40301F09EBDC1EBC10267
:1036500000EB8202D0F8B403526C01F008BD000008
:103660002DE9F0470E46074672B6012936D1234CA4
:10367000214D4022206805F5177105EB8010FDF7FC
:103680005AFA6978A878042202EB012100EB0108BC
:1036900060684FF000094FF0010A012810D1297825
:1036A000284603F097FF00281CBFC4F80490B8F127
:1036B000400F05DDA8F101000AEBA010C5F8740960
:1036C0002068401C2060D5F87409401EC5F87409B4
:1036D000D5F87409002808BFC4E9009AC6EBC600F3
:1036E00007EB80003146D0F8E821D7F8B40301F0A9
:1036F00016FD62B6BDE8F087BC0C00202002002059
:10370000D0F8B40301F042BD70B504460A4611F08A
:10371000800F01F07F0014BFC0EBC001C2EBC201FB
:1037200004EB810114BF383101F5EE7100258D7075
:103730000870D009487094F88003012804BF022063
:1037400070BD012084F88003206802F00CF984F831
:103750008053002070BD70B504468C4611F0800F78
:1037600001F07F00C0EBC00104EB810114BF3831D0
:1037700001F5EE7108705FEADC1C81F801C08A6017
:10378000CB7018BFC8800025022B08BF0D7194F8BC
:103790008003012804BF022070BD012084F880034B
:1037A000206801F0B3FF284684F8805370BD70B5DF
:1037B00004468C4601F07F00C0EBC00104EB8101A0
:1037C0000025C1F8E821C1E97C3581F8DD5181F897
:1037D000DC01206901F5EE71012808BF0A6194F847
:1037E0008003012804BF022070BD012084F88003FB
:1037F000227C20681CF07F0F05D002F019F984F8B4
:103800008053002070BD01F0E3FFF8E770B5044677
:103810000D4611F0800F01F07F0014BFC0EBC00116
:10382000C5EBC50104EB810114BF383101F5EE7120
:1038300001228A700870E809487094F88003012812
:1038400004BF022070BD84F88023206802F0BDF818
:1038500015F07F0F05D1217C04F56172206802F01C
:1038600063F8002084F8800370BD000070B5044642
:103870008C4601F07F00C0EBC00104EB8101002504
:103880004A64C1E91335012381F8393001F8380F52
:103890002069012808BF0A6194F88003012804BF49
:1038A000022070BD84F88033227C20681CF07F0FDA
:1038B00006D002F0BDF800BF84F88053002070BD30
:1038C00001F086FFF8E700002DE9F04F0568044697
:1038D00083B00026284602F016FA00281CBF03B069
:1038E000BDE8F08F206802F037FA002804BF03B06B
:1038F000BDE8F08F206802F02FFA10F0020F04D01C
:103900002068416901F002014161206802F024FA57
:1039100010F4002F4FF008084FF0100A4FF0010B81
:103920004ED0206802F0FAF9070049D017F0010FD5
:1039300043D0F1B2206802F007FA814610F0010F7F
:103940002AD005EB4611C1F808BB2069012811D126
:10395000C6EBC60004EB8000D1F8101BD0F8E421C0
:10396000C1F31201511AC0F8F411D0F8E811114452
:10397000C0F8E811F1B22046FFF772FE2069012875
:1039800002BF002ED4F8F001002805D104F56172C1
:103990000121206801F0C8FF19F0080F06D0204669
:1039A00000F03CFA05EB4610C0F8088B19F0100F38
:1039B0001CBF05EB4610C0F808AB761C7F08B5D1DC
:1039C000206802F0C9F910F4802F75D0206802F049
:1039D0009EF95FEA00094FF000066DD019F0010F63
:1039E0006BD0F1B2206802F0A0F9074610F0010F89
:1039F00028D00121D5F8342801FA06F022EA000087
:103A0000C5F8340805EB4610C0F8081920690128EC
:103A100007D1C6EBC60004EB8000D0E910211144A9
:103A20004164F1B22046FFF711FE2069012802BF70
:103A3000002EE06C002805D104F561720121206898
:103A400001F072FF17F0080F04D005EB46110820B3
:103A5000C1F8080917F0100F04D005EB461110202B
:103A6000C1F8080917F0400F04D005EB46114020BB
:103A7000C1F8080917F0020F04D005EB4611022027
:103A8000C1F8080917F0800F49D020680190C6EBF3
:103A9000C60004EB800000F13808D8E90501471A98
:103AA000D8F80800874288BF0746F81C4FEA900AFA
:103AB000019800EB461B1DE036E030E0471AD8F8CD
:103AC0000800B84238BF0746F81C4FEA900A207C2D
:103AD0000090BBB2F2B2D8F80C10019802F06EF967
:103AE000D8F80C003844C8F80C00D8F8180038444E
:103AF000C8F81800DBF8180980B2504584BFD8E92F
:103B00000501884201D90028D8D147B9019901207F
:103B1000B040D1F8341881430198C0F83418761CAD
:103B20005FEA59097FF45AAF206802F015F910F0E6
:103B3000004F0DD0D5F8040820F00100C5F80408A6
:103B4000204600F051F92068416901F000414161CF
:103B5000206802F001F910F4006F0CD0D5F80808C5
:103B600010F0010F1CBF204600F060F92068416989
:103B700001F400614161206802F0EEF810F4805F0A
:103B80005CD0D5F8040820F00100C5F80408002135
:103B9000206802F087F86068D0B110F001004FF0A3
:103BA000FF021CBFC5F80829C5F8082B61688142CF
:103BB0000ED900BF05EB4011C1F80829C1F8082B48
:103BC000C1F82829C1F8282B6168801C8142F1D8EE
:103BD0004FF0FF30C5F81808D5F81C0840F0011068
:103BE000C5F81C08206B60B1D5F8840840F00B00C4
:103BF000C5F88408D5F8440840F00B00C5F844081F
:103C00000BE0D5F8140840F00B00C5F81408D5F8FF
:103C1000100840F00B00C5F81008D5F8000820F493
:103C2000FE60C5F80008217C04F56172206801F08F
:103C30007BFE2068416901F480514161206802F0F7
:103C40008BF810F4005F1CD0206801F0A7FD2068FD
:103C5000C16821F47051C160206802F037F860B388
:103C60000320E060402060612068C16841F4C051D9
:103C7000C160204600F0A7F82068416901F40051B6
:103C80004161206802F068F810F0100F41D0206800
:103C9000816921F010018161D5F8208008F00F00C2
:103CA000C0EBC00004EB800000F5EE77C8F34340A2
:103CB00002280CD006281CD026E00020E0604FF43B
:103CC000007060612068C16841F41051D0E747F688
:103CD000F07018EA000F17D0C8F30A129046284671
:103CE000F96802F03DF8F8684044F860B86940446B
:103CF00009E0082204F56171284602F031F8B8693C
:103D0000C8F30A110844B8612068816941F01001C4
:103D10008161206802F020F810F0080F07D02046DB
:103D200000F066F82068416901F0080141612068EF
:103D300002F012F810F4801F08D0F1B2204600F013
:103D40003AF82068416901F480114161206802F06D
:103D500003F810F4001F08D0F1B2204600F02FF84D
:103D60002068416901F400114161206801F0F4FF0D
:103D700010F0804F07D02046FFF764FC20684169AF
:103D800001F080414161206801F0E6FF10F0040F6E
:103D900004BF03B0BDE8F08F2068456815F0040F3C
:103DA0001CBF2046FFF7ACFC2068416829434160F6
:103DB00003B0BDE8F08FD0F8B40301F002BAD0F838
:103DC000B40301F000BA10B50446C0680121002810
:103DD00008BF0021D4F8B40301F03AFAD4F8B403D0
:103DE000BDE8104001F002BAD0F8B40301F01DBAEA
:103DF000D0F8B40301F01FBA10B5044690F8800360
:103E0000012804BF022010BD012084F8800320682F
:103E100001F0C3FF002084F8800310BDD0F8B42364
:103E200000F56171104601F01DBA000010B504469E
:103E3000D0F8B40301F04CFA2068D0F8001E41F02D
:103E40000101C0F8001E206A002808BF10BD034809
:103E5000016841F00601016010BD000010ED00E0B6
:103E60002DE9F05F5F4F06468946386801F0FF0A8A
:103E700000F00F00484506D287F800A0386800F02F
:103E80000F00484540D13078574D10F0020F05D053
:103E90002868B16820F0F00008432860307810F0FE
:103EA000010F65D070685149012825D0022818BF3C
:103EB0000328096825D011F0020F65D0296821F088
:103EC000030108432860FFF727FB0446706841F2AE
:103ED0008838012819D0022827D00328286834D030
:103EE00010F00C0F44D000BFFFF716FB001B40453D
:103EF0003AD90320BDE8F09F096811F4003FDDD1F5
:103F000042E011F0007FD9D13EE0286800F00C00BB
:103F100004282DD0FFF700FB001B4045E9D8286896
:103F200000F00C000428F5D122E0286800F00C0015
:103F300008281DD0FFF7F0FA001B4045D9D82868A3
:103F400000F00C000828F5D112E04FF00C0B3BEA12
:103F500000000DD0FFF7E0FA001B4045C9D82868E3
:103F60003BEA0000F6D103E0286810F00C0FBBD14B
:103F7000386800F00F00814509D287F800A0386842
:103F800000F00F00484502D00120BDE8F09F3078D6
:103F900010F0040F05D02868F16820F4E0500843C1
:103FA0002860307810F0080F06D02868316920F4B6
:103FB000604040EAC100286000F04EF82968F02215
:103FC00092FAA2F201F0F001B2FA82F2D140084A6C
:103FD000515CC840074908600F20FFF7C5FA002070
:103FE000BDE8F09F003C0240083802400038024023
:103FF00088AC000898010020084809490068096851
:104000004FF4E05292FAA2F201F4E051B2FA82F2D5
:10401000D140044A515CC84070470000980100201C
:104020000838024088AC0008084809490068096857
:104030004FF4604292FAA2F201F46041B2FA82F2C5
:10404000D140044A515CC8407047000098010020EC
:104050000838024088AC00082048006810F00C01C5
:104060001F4808BF7047DFF87CC0042904BF6046C2
:104070007047082918BF704710B41B4B196801F02E
:104080003F02196811F4800F47F6C0710BD0BCFBDA
:10409000F2F01A680A4091FAA1F1B1FA81F122FA1C
:1040A00001F148430AE0B0FBF2F01A680A4091FAC5
:1040B000A1F1B1FA81F122FA01F1484319684FF4F4
:1040C000403292FAA2F201F44031B2FA82F2D140C7
:1040D000491C4900B0FBF1F010BC704708380240A1
:1040E0000024F4000048E801043802402DE9F84FAC
:1040F00004460078CE4FCF4D10F0010F40D0386805
:1041000000F00C00042809D0386800F00C000828E2
:104110000DD1281D006810F4800F08D0286810F415
:10412000003F2DD06068002800F07F8128E0C24960
:1041300020790870606890B1FFF7EEF906462868AC
:1041400010F4003F1CD100BFFFF7E6F9801BC82820
:1041500000F21581286810F4003FF5D010E0FFF759
:10416000DBF90646286810F4003F09D0FFF7D4F9C0
:10417000801BC82800F20381286810F4003FF5D1A5
:104180002078DFF8B88210F0020F4FF0000958D005
:1041900038684FF0F80A10F00C0F16D0386800F0AD
:1041A0000C00082804D1A648006810F4800F0CD039
:1041B000E06890B30120C8F80000FFF7ADF90646AB
:1041C000286810F0020F13D01BE0286810F0020FCF
:1041D0001CBFE068012840F0288128689AFAAAF1FB
:1041E00020F0F8022069B1FA81F18840104312E012
:1041F000FFF792F9801B02287ED8286810F0020F82
:10420000F6D028689AFAAAF220F0F8012069B2FAEA
:1042100082F290400843286013E0FFE7C8F800905E
:10422000FFF77AF90646286810F0020F09D000BFA0
:10423000FFF772F9801B02285ED8286810F0020F81
:10424000F6D1207810F0080F2ED07E48DFF8F8A1C4
:104250006169A1B101210160FFF75EF90646DAF854
:10426000000010F0020F1FD1FFF756F9801B022843
:1042700042D8DAF8000010F0020FF5D014E0C0F8D0
:104280000090FFF749F90646DAF8000010F0020F37
:104290000AD000BFFFF740F9801B02286FD8DAF878
:1042A000000010F0020FF5D1207810F0040F4FD06D
:1042B0006648016841F0805101600068DFF890A114
:1042C00000F080500090DAF8000040F48070CAF8E6
:1042D0000000FFF721F90646DAF8000010F4807FAD
:1042E0000CD100BFFFF718F9801B022847D8DAF875
:1042F000000010F4807F00E041E0F3D0554E207ABA
:104300003070A06841F2883B88B1FFF705F982461A
:10431000306810F0020F1BD1FFF7FEF8A0EB0A0087
:1043200058452CD8306810F0020FF5D010E0FFF798
:10433000F3F88246306810F0020F09D0FFF7ECF86E
:10434000A0EB0A0058451AD8306810F0020FF5D1DA
:10435000A069E8B3396801F00C01082965D002288A
:10436000C8F860900ED0FFF7D7F80446286810F020
:10437000007F57D0FFF7D0F8001B02284ED903204A
:10438000BDE8F88FFFF7C8F80646286810F0007FF0
:1043900009D000BFFFF7C0F8801B0228EFD82868BB
:1043A00010F0007FF6D1D4E90701014347F6C0724F
:1043B00092FAA2F2606AB2FA82F29040A26A4FF0D8
:1043C000FF3303EB52024FF4403393FAA3F300E0C0
:1043D00028E0B3FA83F39A40104308434FF0706229
:1043E00092FAA2F2E16AB2FA82F2914001431448D1
:1043F00001600120C8F86000FFF78EF804462868C5
:1044000010F0007F0ED100BFFFF786F8001B0228D6
:10441000B5D8286810F0007FF6D003E0286810F0C7
:10442000007FA7D10020BDE8F88F0120BDE8F88FFC
:10443000083802400038024002380240000047427B
:1044400004380240800E474274380240403802402F
:104450000070004070380240002804BF01207047FF
:1044600070B5044690F85100002520B984F85050EA
:10447000204600F037F8022084F8510020680168D7
:1044800021F040010160D4E901010843D4E903129D
:104490001143084361690843218B01F4007108430B
:1044A000E1690843216A0843A16A0843216808605A
:1044B000A069042101EA1040616A0843216848604C
:1044C000A06AB0F5005F02D12168E06A0861206847
:1044D000C16921F40061C1616565012084F8510062
:1044E000002070BD7047704710B5FFF7FCFF10BD8E
:1044F000002804BF0120704710B5044690F8390029
:1045000028B9002084F83800204600F00CF802207A
:1045100084F83900211D206800F074FB012084F824
:104520003900002010BD70470268012303FA01F131
:10453000136A8B431362136A194311620168A1F174
:104540008042B2F5803203D14A6C42F400424A64A0
:104550000068016841F001010160002070470068B7
:1045600081B0016811F0010F04BF016811F0020F62
:1045700003D04068009001B07047016811F0040F4B
:1045800004BF016811F0080FF3D101B070470000BB
:1045900070B5016804460868CA684B6910F00F0FCF
:1045A0004FF0200543D040F2011C13EA0C0F00F03D
:1045B000F18010F0010F18BF12F4807F05D0D4F8FD
:1045C0003CC04CF0010CC4F83CC010F0040F18BF04
:1045D00013F0010F05D0D4F83CC04CF0020CC4F825
:1045E0003CC010F0020F18BF13F0010F05D0D4F833
:1045F0003CC04CF0040CC4F83CC010F0080F18BFCD
:1046000013F0010F03D0E36B43F00803E363E36BA4
:10461000002B08BF70BD10F0200F18BF12F0200F44
:1046200072D094F83A202046222A44D07CE010F040
:10463000200F18BF12F0200F67D094F83A202046C0
:10464000222A18BF70BD8268B2F5805F1ED0026951
:104650005AB3496801F07F02816A4B1C83620A7079
:10466000C18D491E0904090CC18518BF70BD0168C0
:10467000CA6822F49072CA6001684A6922F0010295
:104680004A6180F83A5000F0FDF870BD0369826A13
:104690004968002B14BFC9B2C1F308011180816AB7
:1046A00014BF491C891C8162DAE74A68816A4B1C85
:1046B00083620A70D4E78268B2F5805F0FD0026926
:1046C000E2B1496801F07F02816A4B1C83620A7083
:1046D000C18D491E0904090CC18525D116E0036965
:1046E000826A4968002B14BFC9B2C1F30801118066
:1046F000816A14BF491C891C8162E9E74A68816AA2
:104700004B1C83620A70E3E70EE043E00168CA686D
:1047100022F49072CA6001684A6922F001024A617B
:1047200080F83A5000F0AEF820684169E26BC1F3BE
:10473000801102F00802114326D0C16821F4907163
:10474000C1602068416921F00101416184F83A505B
:104750002068416911F0400F12D0416921F04001F9
:104760004161606B60B12D490165606BFEF738FDFA
:10477000002808BF70BD606B016DBDE87040084740
:104780002046FFF7ECFE70BD2046FFF7E8FE002054
:10479000E06370BD10F0800F18BF12F0800F2CD0B6
:1047A00094F83900212818BF70BDA068B0F5805F6B
:1047B000206A16D0411C2162216800784860E08C94
:1047C000401E0004000CE08418BF70BD2068C16862
:1047D00021F08001C1602068C16841F04001C160E2
:1047E00070BD0088C0F30800486020690028206A76
:1047F00014BF401C801C2062E1E710F0400F14BF82
:1048000012F0400F70BD2046CA6822F04002CA6014
:1048100084F8395000F037F870BD0000994C00085A
:10482000002804BF0120704770B5044690F8390095
:10483000002520B984F83850204600F022F82420C2
:1048400084F839002068C16821F40051C160204615
:1048500000F02AFA2068016921F490410161206882
:10486000416921F02A0141612068C16841F4005189
:10487000C160E563202084F8390084F83A00002004
:1048800070BD704770470068016811F0400F1CBF91
:104890006FF0400101607047FEE7FEE770470000DF
:1048A0000148FFF711B800007808002070477047F2
:1048B0002DE9F04F394D93B00024286840F0805026
:1048C00028602868364E00F080501190306820F43F
:1048D000404040F40040306030684FF0010800F480
:1048E000404011900520CDE9008002277805CDE9F0
:1048F00006704FF01009A820CDE908904FF0040A87
:104900000720CDE90AA06846FFF7F0FB4FF00F0B38
:1049100070B9A814CDE90E40CDE90CB702210CA85E
:104920001094FFF79DFA002804BF13B0BDE8F08F84
:10493000286840F080502860286800F0805011906E
:10494000306820F4404040F400403060306800F4AB
:10495000404011900320CDE90004CDE90389CDE961
:104960000674C020CDF82090CDF82CA0CDE9090721
:104970006846FFF7BBFB78B94FF48050CDE90E4095
:10498000CDE90CB702210CA81094FFF769FA0028B2
:1049900004BF13B0BDE8F08FFEE7000040380240CE
:1049A0000070004038B50024224908283CD2DFE8D6
:1049B00000F0040D161F283B3B311F4C086840F0E7
:1049C00001000860086800F001002BE01B4C08683B
:1049D00040F002000860086800F0020022E0184C75
:1049E000086840F004000860086800F0040019E05E
:1049F000144C086840F008000860086800F00800DF
:104A000010E0114C086840F010000860086800F0E1
:104A1000100007E00D4C086840F08000086008684E
:104A200000F08000009002E009A004F0B3FE2046F0
:104A300038BD00003038024000000240000402404F
:104A400000080240000C024000100240001C02401E
:104A500050696E6D6170206572726F723A20777264
:104A60006F6E6720706F7274206E756D6265722E46
:104A70000000000010B5FEF755FDBDE81040FFF73F
:104A800033BD0000DFF86CC030B4DCF800001A4B16
:104A900010F00C01194806D05C00042908BF04601E
:104AA00002D008290CD00360DCF80010144AC1F3CE
:104AB0000311515C026822FA01F1016030BC7047B9
:104AC00010490A68C2F380550A68002D02F03F02BF
:104AD00014BFB4FBF2F2B3FBF2F20B680968C3F344
:104AE00088135A43C1F30141491C4900B2FBF1F15B
:104AF0000160D9E7083802400024F4009801002042
:104B000034AC00080438024030B5314887B0016841
:104B100041F4700101602F48016841F0010101601A
:104B20002D4A00211160026822F4102222F08072C6
:104B30000260031D294A1A60026822F48022026082
:104B40002748016027495806086028492648086018
:104B50002748016821F007010160016841F0010167
:104B60000160FEF7E7FC2348016841F001010160A4
:104B70000068214D00F00100059001200090019097
:104B800002900220039069462846FEF7BDFB0122F1
:104B900011462846FEF7BAFC184C0121491CA142D7
:104BA000FCDB002201212846FEF7B0FC0220401C5D
:104BB000A042FCDBFFF77CFE1148016841F00801D0
:104BC0000160016821F00801016007B030BD0000FC
:104BD00088ED00E000380240083802401030002420
:104BE0000C38024008ED00E00024F4009801002099
:104BF000003801403038024000000240A086010029
:104C00002038024070B402681F4BDFF880C0204C8F
:104C1000204D984218BFB0F1804F04D060451CBFB2
:104C2000A042A84203D14E6822F07002324398425B
:104C300018BFB0F1804F14D0604518BFA04210D00B
:104C4000A8421CBFA0F1804CBCF5A03C09D0A0F14B
:104C5000804CBCF5A23C1CBFA0F1804CBCF5A43C30
:104C600005D1D1F80CC022F440724CEA0202026075
:104C70008A68C2620A688262984204BF0969016355
:104C80000121416170BC70470000014000040040F8
:104C900000080040000C004010B5806B0021C18569
:104CA000C184FFF75CFC10BD2DE9F04104460068AB
:104CB0000169E26821F44051114301612068C16833
:104CC0002369A268D4F81CC01A43636921F40371F4
:104CD00043EA0C0321F414411A431143C1602068D4
:104CE0004169A26921F4407111434161E2693226B0
:104CF000B2F5004FBA48BB49BB4D22685DD08A422D
:104D000018BF824240F01281FFF78EF900EBC0011C
:104D100001EB001061688900B0FBF1F7FFF784F93F
:104D200000EBC00101EB001061688900B0FBF1F0FD
:104D3000A5FB001040096FF01801484307EB800005
:104D400006EB0010A5FB0010400900F0F007FFF78C
:104D50006BF900EBC00101EB001061688900B0FB4A
:104D6000F1F0A5FB0010400907EB0017FFF75CF915
:104D700000EBC00101EB001061688900B0FBF1F8A5
:104D8000FFF752F900EBC00101EB001061688900E8
:104D9000B0FBF1F0A5FB001040096FF0180148438B
:104DA00008EB800006EB0010A5FB00102168C0F3A3
:104DB000431038448860BDE8F0818A4218BF8242BF
:104DC00059D1FFF731F900EBC00101EB0010616828
:104DD0004900B0FBF1F0A5FB001040090701FFF707
:104DE00023F900EBC00101EB001061684900B0FB42
:104DF000F1F8FFF719F900EBC00101EB0010616851
:104E00004900B0FBF1F0A5FB001040096FF018015C
:104E1000484308EB800006EBC000A5FB00104009EA
:104E200000F0F80007EB4007FFF7FEF800EBC001C9
:104E300001EB001061684900B0FBF1F8FFF7F4F8EE
:104E400000EBC00101EB001061684900B0FBF1F01C
:104E5000A5FB001040096FF01801484308EB8000E3
:104E600006EBC000A5FB00102168C0F342103844D7
:104E70008860BDE8F081FFF7BFF800EBC00101EBEF
:104E8000001061684900B0FBF1F0A5FB001040097B
:104E90000701FFF7B1F800EBC00101EB00106168FA
:104EA0004900B0FBF1F8FFF7A7F800EBC00101EBF8
:104EB000001061684900B0FBF1F0A5FB001040094B
:104EC0006FF01801484308EB800006EBC000A5FB1B
:104ED0000010400900F0F80007EB4007FFF78CF8DE
:104EE00000EBC00101EB001061684900B0FBF1F874
:104EF000FFF782F800EBC00101EB00106168490088
:104F0000B0FBF1F0A5FB001040096FF01801484319
:104F100008EB800006EBC000A5FB00102168C0F381
:104F2000421038448860BDE8F08100BFFFF764F8A4
:104F300000EBC00101EB001061688900B0FBF1F7E4
:104F4000FFF75AF800EBC00101EB0010616889001F
:104F5000B0FBF1F0A5FB001040096FF018014843C9
:104F600007EB800006EB0010A5FB0010400900F0E5
:104F7000F007FFF741F800EBC00101EB001061689A
:104F80008900B0FBF1F0A5FB0010400907EB00170A
:104F9000FFF732F800EBC00101EB001061688900F7
:104FA000B0FBF1F8FFF728F800EBC00101EB0010AF
:104FB00061688900B0FBF1F0A5FB001040096FF0BB
:104FC0001801484308EB800006EB0010A5FB001019
:104FD0002168C0F3431038448860BDE8F0810000C8
:104FE00000140140001001401F85EB5110B5D0F8AE
:104FF000142252689047002010BD134610B50A468F
:10500000002100F0ECF8002010BD134610B50A4650
:10501000002100F066F9002010BD10B50521002325
:10502000C0F8F4111A46194600F0D9F8002010BD56
:1050300010B502238261C0F8F431C26113460A46FA
:10504000002100F04EF9002010BD10B5042100230E
:10505000C0F8F4111A46194600F043F9002010BDBB
:1050600010B5D0F82002FEF74FFB002010BD70B540
:105070001346044659B1D4F814024269002A4CD0B0
:1050800094F8FC01032804BF2046904745E0D4F87B
:10509000F411002504F11400022938D1D0E90221CD
:1050A0008A420DD9511A81608AB219462046FFF70B
:1050B000ACFF00231A461946204600F090F826E07F
:1050C0004068B0FBF1F201FB12029AB9884211D399
:1050D000D4F8F81188420DD2002211462046FFF77D
:1050E00094FF00231A4619462046C4F8F85100F0F0
:1050F00076F80CE0D4F81402C16829B194F8FC01E8
:10510000032804BF204688472046FFF786FF94F80F
:105110000002012808BF84F80052002070BD70B55D
:105120001546044651B1D4F81402826952B394F87A
:10513000FC01032804BF2046904723E0D4F8F41173
:1051400004F5827003291DD1D0E902C39C450CD916
:10515000ACEB03038360C068984298BF03469AB2E1
:1051600029462046FFF749FF0CE0D4F814020169F4
:1051700029B194F8FC01032804BF20468847204643
:10518000FFF763FF002070BD0020704710B50121BC
:1051900080F8FC11D0F81422017952689047002061
:1051A00010BD11F0800F01F07F01D0F82002C1EB9B
:1051B000C10100EB810014BF90F83A0090F8DE01C5
:1051C0007047002070470020704710B59C4613467A
:1051D000D0F820026246FEF7BEFA002010BD10B5DE
:1051E000D0F82002FEF7E3FA002010BD70B50022CF
:1051F000044640231146FFF7E8FF40252B460022D6
:1052000080212046C4F81051FFF7DFFF01202562FE
:1052100084F8FC01D4F8180228B1D4F814022179DA
:10522000426820469047002070BD90F8FD1180F83C
:10523000FC110020704710B590F8FC11032905D12E
:10524000D0F81412C969002918BF8847002010BD82
:1052500001740020704710B5D0F82002FEF7CCFD95
:10526000002010BD10B5044600F5027000F040F8B3
:105270000120C4F8F401B4F80E02C4F8F80194F85F
:10528000080210F01F010AD001290ED0022912D005
:1052900000F08001204600F014F8002010BD04F555
:1052A0000271204600F044F8F7E704F50271204649
:1052B00000F00BFAF1E704F50271204600F080F9E6
:1052C000EBE710B5D0F82002FEF7A0FA002010BDE1
:1052D00090F8FC1180F8FD11042180F8FC110020E9
:1052E000704710B5D0F82002FEF7C0FA002010BDBC
:1052F0000A7802704A7842708A78CB7802EB0322EF
:1053000042800A794B7902EB032282808A79C9793B
:1053100002EB0121C180704710B5D0F8142202249D
:1053200022B112689047002808BF0024204610BD13
:10533000F8B50D46497800260A2980F0F180DFE8AB
:1053400001F0FAF9EFF8EF8505EFE3A40446688869
:10535000010A082980F0C380DFE801F0C1040C1EB7
:10536000C1C1555FD4F81012207C0A686946904785
:1053700001465DE0207C0028D4F8140205D0C16A03
:10538000684688470146022051E0816A684688479E
:105390000146022048704BE0C0B2062874D2DFE814
:1053A00000F0030B131B232BD4F81012207C4A6847
:1053B0006946904701463BE0D4F81012207C8A6889
:1053C00069469047014633E0D4F81012207CCA6841
:1053D0006946904701462BE0D4F81012207C0A69F8
:1053E00069469047014623E0D4F81012207C4A69B0
:1053F0006946904701461BE0D4F81012207C8A6968
:105400006946904707E0207C002868D1D4F8140250
:10541000416B6846884701460AE0207C00285ED13F
:10542000D4F81402016B684688470146072048708B
:10543000BDF8000000281CBFEA88002A57D082422D
:1054400088BF0246ADF8002020467AE00446A888CE
:10545000002804BFE888002841D1A87800F07F0523
:1054600094F8FC0103283AD084F8FE5129462046DE
:10547000FFF7F1FE2046FFF7E8FD002D0CBF0120ED
:10548000022084F8FC0132E029E0A9784B4D044663
:105490000129297023D894F8FC01022802D003289E
:1054A0000ED01CE041B10320616084F8FC0120466D
:1054B000FFF732FF022812D02046FFF7C6FD16E0A4
:1054C000B9B160688842F7D0C1B22046FFF78EFDBF
:1054D000297820466160FFF71FFF0228ECD1802168
:1054E0002046FFF7EEFE00212046FFF7EAFE304699
:1054F000F8BD022084F8FC0120466160FFF776FDCC
:105500002046FFF7A2FDF2E7E988012908D190F8CB
:10551000FC11022910D0032904BF0122011D10D063
:1055200004468021FFF7CDFE00212046FFF7C9FE8B
:10553000DDE71BE02AE007E000218160012200F1A5
:105540000801FFF775FDD2E790F8FC11022918BF9A
:105550000329E5D10121C160D0F8041200291CBF44
:105560000321C160022200F10C01EAE704466888C9
:1055700029460128BBD1C4F80402D4F81402826879
:10558000204690472046FFF760FDB0E7044690F8BC
:10559000FC012946022818BF0328A0D14888012809
:1055A000A5D10020C4F80402D4F814028268204671
:1055B00090472046FFF749FD99E7000028020020A8
:1055C00070B50D46044628780026097900F0600081
:1055D000202807D06878002848D0012828D0032840
:1055E00008D051E0D4F8140229468268204690473A
:1055F000002070BD94F8FC01022802D0032805D0D9
:105600003AE0002918BF802943D13DE0688828B9D5
:1056100000291EBF80292046FFF753FED4F814024C
:1056200029468268204690472046FFF70EFD2BE072
:1056300094F8FC01022802D0032805D01CE00029C0
:1056400018BF802925D11FE06888E8B911F07F0FC5
:1056500008D02046FFF704FDD4F8140229468268DA
:10566000204690472046FFF7F0FC0DE094F8FC013F
:1056700002280BD0032810D080212046FFF721FEFE
:1056800000212046FFF71DFE304670BD11F07F0F50
:10569000FAD02046FFF715FEF6E701F07F0011F083
:1056A000800F04EB001014BF00F1140500F58275A3
:1056B0002046FFF776FD002818BF0120022228604F
:1056C00029462046FFF7B4FCDEE770B5044690F8A3
:1056D000FC010D4603280ED1287901280BD8D4F8F7
:1056E0001402826820469047E888002804BF2046BC
:1056F000FFF7ABFC07E080212046FFF7E2FD002129
:105700002046FFF7DEFD002070BD00004B7801222F
:1057100091F800C002FA0CF2012BD0F81C380CD022
:1057200043EA0242C0F81C280A7800EB4210D0F885
:10573000002B12F4004F20D02CE092B21A43C0F894
:105740001C280A7800EB4210D0F8003913F4004FFF
:1057500020D1D0F80039B1F808C0CCF30A0C43EAE4
:105760000C03C978890441EA8251194341F400418C
:1057700041F08051C0F800190CE0D0F8002B0B89E3
:10578000C3F30A031A43C978034B43EA8141114327
:10579000C0F8001B0020704700800010D0F80019EE
:1057A0006FF30A01C0F80019D0F8081801F00601DB
:1057B000042905D1D0F8001941F00301C0F80019FF
:1057C000D0F8041841F48071C0F804180020704724
:1057D00010B491F801C00B7800EB4313BCF1010F3A
:1057E0002BD0D3F810CB6FF3120CC3F810CB0B787F
:1057F00000EB4313D3F810CB6FF3DC4CC3F810CBA2
:105800004B69002B1CBF8B684B610B7800EB43137B
:10581000D3F810CB4CF4002CC3F810CB0B7800EB72
:105820004313D3F810CB8C68C4F312044CEA040C75
:10583000C3F810CB012A6BD164E0D1F814C0BCF1DD
:10584000000FD3F810C941D06FF3120CC3F810C980
:105850000B7800EB4313D3F810C96FF3DC4CC3F89B
:1058600010C9D1F814C08B689C4598BF63464B6142
:105870000B7800EB4313D3F810C94CF4002CC3F899
:1058800010C90B7800EB4313D3F810C94C69C4F36B
:1058900012044CEA040C00BFC3F810C9012A2AD034
:1058A0004A694AB1D0F834280B784FF0010C0CFA51
:1058B00003F31A43C0F83428097800EB4110D0F8FC
:1058C000001941F00441C0F800192AE06FF3DC4CE4
:1058D000C3F810C90B7800EB4313D3F810C94CF48C
:1058E000002CC3F810C90B7800EB4313D3F810C990
:1058F0006FF3120CD0E70B7800EB43130A69C3F87F
:105900001429D9E70B7800EB4313CA68C3F8142BAA
:10591000097800EB4110D0F8001B41F00441C0F8B9
:10592000001B002010BC70470023C0F8103BD0F8CB
:10593000103B43F40023C0F8103BD0F8103B43F079
:105940001803C0F8103BD0F8103B43F0C043C0F838
:10595000103B012905D1C0F8142B4FF08021C0F86D
:10596000001B002070474B780A7800EB4212012B95
:105970000BD0D2F8003B23F40013C2F8003BCA78E6
:10598000032A18BF022A15D01DE0D2F8003923F4EB
:105990000013C2F80039CA78032A18BF022A12D1AC
:1059A000097800EB4110D0F8001941F08051C0F89F
:1059B000001908E0097800EB4110D0F8001B41F015
:1059C0008051C0F8001B002070474B780A7800EB2C
:1059D0004212012B05D0D2F8003B13F0004F15D036
:1059E0001AE0D2F8003913F0004F05D1D2F800398F
:1059F00023F08043C2F80039097800EB4110D0F859
:105A0000001941F40011C0F800190EE0D2F8003B73
:105A100023F08043C2F8003B097800EB4110D0F836
:105A2000001B41F40011C0F8001B0020704700006B
:105A300030B44C786FF0604C0B7800EB4313012CC2
:105A400032D0D3F8104B6FF31204C3F8104B0B781D
:105A500000EB4313D3F8104B6FF3DC44C3F8104B47
:105A60004B69002B7ED08C6823445B1EB3FBF4F3A0
:105A70009BB20C7800EB4414D4F8105B0CEAC34CD6
:105A800045EA0C0CC4F810CB91F800C000EB4C1C9C
:105A9000DCF8104B8D686B43C3F312032343CCF83F
:105AA000103B012A7ED1D7E04C697CB3D3F8104972
:105AB0006FF31204C3F810490B7800EB4313D3F8CB
:105AC00010496FF3DC44C3F810494C698B681C44DF
:105AD000641EB4FBF3F30CEAC34C0B7800EB4313E6
:105AE000D3F810494CEA040CC3F810C90B7800EB4A
:105AF0004313D3F810C94C69C4F312044CEA040CE4
:105B0000C3F810C9CB78012B18D029E0FFE7D3F8F0
:105B100010C96FF3DC4CC3F810C90B7800EB4313CA
:105B2000D3F810C94CF4002CC3F810C90B7800EB63
:105B30004313D3F810C96FF3120C0FE00B7800EB8E
:105B40004313D3F810C92CF0C04CC3F810C90B781C
:105B500000EB4313D3F810C94CF0005CC3F810C934
:105B6000012A00E062E021D0CB78012B26D04B69DE
:105B70006BB1D0F8343891F800C0012404FA0CFC61
:105B800043EA0C03C0F83438CB78012B16D00B78DD
:105B900000EB4313D3F800C94CF0044CC3F800C920
:105BA000CB7800E05EE0012B68D118E091F800C0EE
:105BB00000EB4C1C0B69CCF81439E5E7D0F8083839
:105BC00013F4807F0B7800EB4313D3F800C90CBFAC
:105BD0004CF0005C4CF0805CC3F800C9D7E791F84A
:105BE00000C0CB68898A89B2FAB9C91C8A0845D035
:105BF00012F0010106D053F8045B00EB0C3404F5FD
:105C00008054256091423CBF00EB0C3000F5805081
:105C100034D200BF53F804CBC0F800C053F804CB13
:105C2000C0F800C0891C9142F4D327E00B7800EB48
:105C30004313D3F810CB8C68C4F312044CEA040C61
:105C4000C3F810CB0B7800EB4313D3F810CB4CF414
:105C5000002CC3F810CB24E70B7800EB4313CA6881
:105C6000C3F8142BCA78012A0BD0097800EB411035
:105C7000D0F8001B41F00441C0F8001B002030BCEC
:105C80007047D0F8082812F4807F0A7800EB42129F
:105C9000D2F8003B14BF43F0805343F00053C2F8E6
:105CA000003BE2E70022202343EA8111016106491B
:105CB000521C8A4201D903207047036913F0200F58
:105CC000F6D1002070470000400D03000021D0F8FD
:105CD000082812F0060F14D0D0F8082802F00602A7
:105CE000022A0DD0D0F80828062333EA020207D092
:105CF000D0F8080800F00600042808BF022100E0E0
:105D0000032108467047406900F001007047D0F851
:105D10001818D0F81C08084080B27047D0F818183E
:105D2000D0F81C080840000C7047D0F81028D0F8B4
:105D30003438CB4003F0010342EAC31200EB4110B8
:105D4000D0F808091040704700EB4111D1F8081B4A
:105D5000D0F81408084070474169806908407047CE
:105D60000346D01C820816D012F0010003F58053C0
:105D700003D0D3F800C041F804CB90420BD200BF4F
:105D8000D3F800C041F804CBD3F800C041F804CBED
:105D9000801C9042F4D308467047D0F8002822F4C3
:105DA000FE62C0F80028D0F800284FF4FE6303EA32
:105DB00001111143C0F8001800207047DDF800C041
:105DC000BCF1000F19D1DB1C5FEA930C15D01CF05D
:105DD000010300EB023000F5805002D051F8042B93
:105DE0000260634509D200BF51F8042B026051F8EC
:105DF000042B02609B1C6345F6D300207047FEE72E
:105E000070B50C460546FDF769FA084AF3211160A2
:105E100002210420FDF73EF90023224629461846B8
:105E2000FDF7FAF9BDE87040FDF7ECB90C3C024013
:105E3000002A18BFB0F5A37F24BF4FF0FF30704792
:105E400070B50E460D4900EB4000154651F8204054
:105E500060B2B0F1FF3F07D0094804F0030200210F
:105E60000260084803F0A4F8C4F307212B46324629
:105E7000044802F051FE002070BD0000F4AC0008A0
:105E8000B402002040160020002A18BFB0F5A37FFE
:105E900024BF4FF0FF30704770B50E46114900EB3C
:105EA000400001EB8000154604688088C0F307209D
:105EB000012804BF4FF0FF3070BD60B2B0F1FF3F6A
:105EC00007D0094804F0030200210260074803F0EC
:105ED0006FF8C4F307212B463246044802F0DAFE7D
:105EE000002070BDF4AC0008B40200204016002071
:105EF00010B5054802F084FF00221146024803F065
:105F000057F8002010BD00004016002010B11028E6
:105F100000D811B94FF0FF3070472DE9F04F894696
:105F20002DED048BD1B080464FF4887102A8FAF7AA
:105F300079FE0026B8F1000F7EDDDFF858B3F5EEEC
:105F4000008A9FEDD59A10279FEDD48AC6EB0610E4
:105F500000EB800009EB8004052202A90B20FFF76B
:105F600067FF9DF80800002869D0102867D89DF8C1
:105F70000C5065859DF80BA005F1100202A90420C4
:105F8000FFF756FF2A4602A904F12C00FAF718FE83
:105F900002A9485D20710A2851D2C14A135C1BF83E
:105FA0000000C04A207394F804C052F82020BE4874
:105FB00050F82C00104420604819227B4179112BA5
:105FC00000EE101AB94901EB8201B8EE400AD1ED9A
:105FD000000A30EE200A84ED060A18BF102B34D0D8
:105FE000202B00F0258100216171617384ED068A08
:105FF00084ED078A84ED088A84ED098AA173216102
:1060000021758379C27990F809C003EB0222037AE3
:106010001B0403EB0C631A44521AA5498969114405
:10602000A160817AC07A01EB0020208500210B203D
:1060300000F028FF761C00E001E0464586DB51B009
:106040003046BDEC048BBDE8F08F0AF00701012952
:106050003ED0052908BF677137D0072914BF00213A
:106060001121617118BF4FF0000E2ED0677390F9A7
:106070000210112B00EE101AB8EEC00A20EE280A0A
:1060800084ED070A90F9031000EE101AB8EEC00A6A
:1060900020EE280A84ED080A90F9041000EE101A88
:1060A000B8EEC00A20EE280A84ED090A0EBF0321CB
:1060B00080498978A17341780909CA1F062A78D2D4
:1060C000DFE802F00B0D0F1113154FF0010ECDE7B5
:1060D000012161714FF0000EC8E7022208E004229E
:1060E00006E0082204E0276103E0202200E04022CD
:1060F00022614278C2F3420CBCF1010F08BF0122B9
:1061000059D0BCF1020F08BF022254D0BCF1030FDA
:1061100008BF03224FD0BCF1040F1ABF0022227522
:10612000042248D0A27B032A47D0022A04BF226956
:10613000402A47D000224D92102B45D07222009267
:106140005FF00102A1F1060ABAF1060F64D8002A35
:1061500062D005EB4E05C1EB450ACDF81CA11AF142
:10616000070F48D04D1CA1F1010A05FA0AF5DDF828
:1061700034A1A1F1040ECAF1040A0AFA0EFA554438
:10618000B5FBF2FE479D07EB8C0C05F1060A4D9D11
:106190006D4201EB4501BAFBF1F501FB15A1491C6C
:1061A00001FB0CF1B1FBF2F1009A7244114434E0AE
:1061B000FFE700229CE72275B4E72269202A18BF76
:1061C000402AB7D10122B6E73A4A9278012A0ED086
:1061D000022A08D0032A0CBF4022002200920CBFE2
:1061E00001220022AEE7202200920222AAE710221A
:1061F00000920422A6E701F1010CA1F1010A0CFAB8
:106200000AFC4FF0030A091F0AFA01F16144B1FBCD
:10621000F2FEA901A031C5E70021112B7FF4F1AEF8
:1062200094ED060A30EE490A84ED060AE9E600BF5D
:106230000AF0070101292BD0052908BF677105D095
:1062400007291ABF00216171112121D0202161731A
:1062500084ED078A174984ED088A84ED098A9FED49
:10626000171ADFED170A4A79A27340EE010AC968CE
:106270009FED141A00222161227520EE011A0E4AA8
:10628000B2FBF1F141EE000A1439C4ED060AB8E69A
:106290006171DBE74A0C002000000CC2000000C363
:1062A000DCAC000848020020540C00205002002002
:1062B000401600203002002040600A00287EC43FC3
:1062C00000007042A69B443BF8B500210698089C4C
:1062D000C6B2C3F30745C3F307270091082E08BFD2
:1062E000002D1FD0A819082822D83946234802F0CB
:1062F00025FE0121B140491EA9408DF80000C9B218
:1063000004FA05F28DF80110D2B288438DF802200C
:10631000114040EA01028DF803203946174802F087
:1063200047FE25E0E2B23946144802F041FE1FE084
:1063300005BBFEB1202E1DD8F01DC308002B12DDB9
:106340000DF1FF3013F0010F02D000F8014F2412BD
:106350005A1008D044704FEA242C00F802CF4FEABC
:106360002C24521EF6D16A463946044802F092FCAB
:106370000020F8BD4FF0FF30F8BD000040160020AF
:1063800010B580220021034802F012FE02490020CD
:10639000086010BD40160020B402002038B5044645
:1063A000694640F2211000F001FD00281CBF4FF0AB
:1063B000FF3038BD00982060002038BD0A2824BF77
:1063C0004FF0FF3070472DE9F05FDFF8E881DDE93D
:1063D0000AC112F0FF0708F114094FF0000E18D09F
:1063E000C2F3072ABAF1020F80F0DF800CF0FF053C
:1063F000012D08BF704E03D0022D14BF6F4E704E9A
:10640000704C082D43D2DFE805F0420B0D0F11143C
:10641000171A08F800E049F820E00020BDE8F09FD6
:10642000694A0EE0694A0CE022460AE04FF2244233
:1064300007E047F6E01204E043F6F04201E041F6DF
:10644000786293460BEBDB7B03EB6B0B06EBD676AC
:10645000BBEB660F7CDCB2F1FF3F08BF224602EBCC
:10646000D2727410A3EB62026442A24270DB584AFB
:106470000226584C12F800B0574ABBF1100F0AD050
:10648000BBF1110F46D0BBF1200F62D08DE04FF071
:10649000FF32A346D6E7002D08BF66F3070C00299C
:1064A00008BF08210CF0FF0CBCF1030F1CBFBCF1AE
:1064B000020FBCF1010F78D1022918BF042907D0BF
:1064C000082918BF102903D0202918BF40296CD1F2
:1064D00008F80070BAF1000F14BF012500252554FB
:1064E00049F8203082F802C001F07E00D070BCF183
:1064F000030F08D0BCF1020F08BF402907D000BF2E
:1065000082F804E04EE0202918BF4029F8D101208C
:10651000107147E0002D04BF032262F3070C00292D
:1065200008BF7E210CF0FF02032A08BF31F07E0273
:106530003BD108F80070BAF1000F14BF012200220D
:106540002254264A49F8203001F07E01115429E0F6
:106550002BE0002D08BF66F3070C002908BF4FF49D
:106560007A410CF0FF0CACF10105072D1DD21C4E39
:10657000A1F5FA75B54218D208F80070BAF1000F0B
:1065800014BF01250025255449F8203082F805C0A4
:10659000D160DDE90E0150EA010303D00C9B1370BA
:1065A000C2E904010020BDE8F09F4FF0FF30BDE8D4
:1065B000F09F0000400C0020E0C81000481D0E00B5
:1065C00040420F0048E8010020A1070090D00300DE
:1065D000DCAC00084A0C00203002002058020020E9
:1065E0009DCE03000FB4022805D29DF8101001299A
:1065F00018BF022903D04FF0FF3004B070470E4B94
:106600009DF804201A541233029A43F8202003F113
:1066100008029DED030A02EB800282ED000AA3F15D
:106620000E0211540599002918BF0121034A115483
:10663000002004B07047000036020020380200201D
:1066400001494870002070473002002030B490F8B3
:1066500050104A1E102A16D2DFF858C00022002916
:106660008CF8501023DD00BF02EB8203C45C032CC6
:1066700009D819188D78032D05D1CD780F2D9CBF21
:106680004D78032D03D930BC4FF0FF3070470CF824
:10669000034063448C789C70CC78DC704C785C70E0
:1066A000097919719CF85010521C9142DCDC30BC05
:1066B000002070476002002010B50621AC2000F0D9
:1066C000E1FB0721AD2000F0DDFB0721AE2000F04B
:1066D000D9FB1721A92000F0D5FB5521AB2000F0F4
:1066E000D1FB4221AA2000F0CDFB07219B2000F026
:1066F000C9FB06219C2000F0C5FB0321962000F079
:10670000C1FB3D4C607840B10321902000F0BAFB02
:106710000421912000F0B6FB07E00121902000F059
:10672000B1FB0221912000F0ADFB607840B1032164
:10673000CA2000F0A7FB0421CB2000F0A3FB07E058
:106740000121CA2000F09EFB0221CB2000F09AFB21
:106750000121802000F096FB40F6FE71812000F0C0
:1067600091FB07217F2000F08DFB0121E42000F048
:1067700089FB0121592000F085FB0421E32000F072
:1067800081FB0121E52000F07DFB0121E72000F0E5
:1067900079FB0221E82000F075FB0A21EA2000F0D5
:1067A00071FBFF21EF2000F06DFB8021F82000F04D
:1067B00069FB40F2DC51B72000F064FB0121C420EA
:1067C00000F060FB607840B10321B82000F05AFB74
:1067D0000421B92000F056FB07E00121B82000F0A9
:1067E00051FB0221B92000F04DFB0221BDE8104011
:1067F000F12000F047BB0000300200202DE9F84FE7
:10680000DFF80CB1B1F100090BF1100682464FF030
:10681000000406F1100706F1200852DD04F1A00182
:106820004FF4977000F02EFB012004F0A7F86946A2
:106830004FF48F7000F0BAFA012004F09FF804EBD7
:106840000A0500980BF8050004F1A8014FF49770B1
:1068500000F018FB012004F091F869464FF48F70A6
:1068600000F0A4FA012004F089F80098705504F1B2
:10687000B0014FF4977000F005FB012004F07EF8A2
:1068800069464FF48F7000F091FA012004F076F819
:106890000098785504F1B8014FF4977000F0F2FABF
:1068A000012004F06BF869464FF48F7000F07EFA17
:1068B000012004F063F80098641C08F80500A14565
:1068C000ACDC9BF805008BF80000737933707979A4
:1068D000397098F8052088F800208BF80100737053
:1068E000797088F801208BF80200B370B97088F8CD
:1068F00002208BF80300F370F97088F803208BF8FE
:1069000004003371397188F80420BDE8F88F000065
:106910007C0C00200FB400202DE9F04FD3B00746C7
:106920009DF87CB14490BBF1020F80F02F82FE48AD
:1069300010F80B00002800F02982FC4810F80B002A
:10694000002800F023829DF87481B8F1000F1CBF6D
:10695000B8F1010FB8F1020F40F018829DF87E01E6
:106960009DF886114F904B919DF884619DF87F4171
:10697000BDF88C91102803D0202823D000F006BA4F
:10698000032C1CBF022C012C40F0008260980228CE
:1069900018BF042808D0082818BF102804D02028C1
:1069A00018BF402840F0F281012E18BF022E04D0FB
:1069B000032E18BF042E40F0E981B9F1FF0F00F259
:1069C000E5810EE0481EC82880F0E0816098A0F5BF
:1069D000FA71D748884240F2D981B9F1FF0F00F22D
:1069E000D581DFF850A39AF85000401E10F0FF0543
:1069F00018BF9DF97D110AD005EB8500504490F930
:106A00000400884203DD681E10F0FF05F4D1CA4976
:106A1000AF2000F0CBF9C949B02000F0C7F9C84950
:106A2000B12000F0C3F9C749B32000F0BFF905EB6E
:106A30008500C0494E900844BBF1000F90F803A0B8
:106A40001ED0C14810F90A10BB2000F01BFABF4845
:106A500010F90A10BC2000F015FAB6494E98095CEE
:106A6000C12000F00FFABA4809F1100A4FF0100CDB
:106A7000017843F6095001290FD0022919D025E0E9
:106A8000B44810F90A10BB2000F0FCF9B24810F924
:106A90000A10BC2000F0F6F9DFE7B0495C9A5C9B75
:106AA000B2FBF1F24492B3FBF1F201FB1231490265
:106AB0000AE0AB495C9A5C9BB2FBF1F24492B3FBF7
:106AC000F1F201FB12310902B1FBF0F74498C3B2B5
:106AD000380A8DF800308DF801008DF80270B8F199
:106AE000010F10D19F495E988969401AA0F2DC50CD
:106AF000010E8DF80310010C8DF80410010A8DF8B9
:106B000005108DF806009DF87C11202000EA411B3D
:106B1000BDF88C11DDF83CE1CAB29DF88A71002005
:106B2000BDF88811BEF1100F04D0BEF1200F6ED059
:106B300000F02CB905F00F054BEA05058DF807505C
:106B4000609D8DF80800102D08BF0A2515D00CDCBB
:106B5000022D08BF072510D0042D08BF08250CD032
:106B6000082D08BF092508D009E0202D08BF0B25F6
:106B700003D0402D08BF0C2501D18DF80950012EFE
:106B800004BF9DF8095045F0100514D0022E04BF33
:106B90009DF8095045F020050DD0032E04BF9DF847
:106BA000095045F0300506D0042E04BF9DF8095069
:106BB00045F0400501D18DF809502FB99DF80950D5
:106BC00045F080058DF809508DF80A20012C08BF8A
:106BD000022208D0022C08BF012204D0032C08BFD7
:106BE0008DF80B0001E08DF80B209DF88B21012A18
:106BF00005D19DF80B2042F004028DF80B20032CE8
:106C000006D0022C04BF609A402A06D00BE039E07F
:106C1000609A202A18BF402A05D19DF80B2042F027
:106C200008028DF80B209DF88521012A05D19DF8D9
:106C30000B2042F010028DF80B20002908BF06211E
:106C400003D0042938BF042101D2ADF8881189B2DC
:106C50000A0A8DF80C208DF80D108DF80E008DF8B5
:106C60000F0003F03F008DF80000012C08BF40F03A
:106C7000800004D0032C08BF40F040003DD18DF8C7
:106C800000003AE005F00F0C8DF808004BEA0C0C00
:106C90004B984CF0100C8DF809008DF807C08DF85A
:106CA0000A20002F14BF0020022040F009008DF8B8
:106CB0000B00002908BF052003D0032938BF03209B
:106CC00001D2ADF88801BDF888018DF81020010AC5
:106CD0008DF80C108DF80D00234960984FF0110CC1
:106CE000B1FBF0F0010A8DF80E108DF80F0003F0E3
:106CF0007F008DF800000AF1010A0DEB0C004A46F6
:106D00000DF5C771F9F717FF002140F2451000F0AB
:106D1000B9F80021052000F0B5F81FFA8AF269469B
:106D20000620FFF7B1F821E03802002036020020EB
:106D30009DCE030060020020300C0020340C0020A7
:106D4000380C00203C0C00209C0C0020AC0C0020D7
:106D50003A0200207C0C00208C0C002080841E0055
:106D600000093D00401600200048E801B8F1000F7E
:106D700004BF0121B42010D0B8F1010F04BF0121DC
:106D8000B5200AD0B8F1020F0AD000BF4FF0FF3093
:106D900053B0BDE8F00F5DF814FB00F073F803E0AA
:106DA0000121B62000F06EF80020F1E72DE9F8434C
:106DB0000F46314900EB400001EB8000D0E900456F
:106DC00060B2B0F1FF3F07D02C4804F0030200216D
:106DD00002602B4802F0ECF800200646C4F3074896
:106DE000EDB2009008EB050008281BD8C4F307217A
:106DF000234802F0A3F8C5F108018DF80000A1EBCB
:106E000008029040C0B2220E8DF80100012A12BF84
:106E1000C8409DF9010008418DF8020018BFC0B2BA
:106E200038601EE0B8F1000F1BD1D5B1202D18D865
:106E3000E81D4FEAD008C4F3072143466A461048CC
:106E400001F06AFEB8F1010058BF694604D40A5C3B
:106E5000401E02EB0626FAD5200E012818BF3E6020
:106E600002D00020BDE8F883C5F1200006FA00F149
:106E700041FA00F03860F4E7F4AC0008B4020020F6
:106E800040160020B0F5A37F24BF4FF0FF307047BD
:106E9000F0B50C461B4983B010B1012808D00AE0B8
:106EA00004F003020A600021174802F081F826E08E
:106EB00014F0010F23D1154A00EB400002EB8000D3
:106EC000D0E900568768C6F30720012802BF4FF0BB
:106ED000FF3003B0F0BD68B2B0F1FF3F06D005F05F
:106EE00003020A600021084802F062F800960022BE
:106EF000CDE901742B4611461046FFF7E5F903B0C2
:106F00000020F0BDB402002040160020F4AC0008C0
:106F10002DE9F84F012631461220FFF7B3FF01217A
:106F20001320FFF7AFFFF74C04F1080001F06DFCF0
:106F3000E169401AA0611F214D20FFF7A3FF002146
:106F40004C20FFF79FFFF04CAF202168FFF79AFF1E
:106F5000B0206168FFF796FFB120A168FFF792FFAC
:106F6000B320E168FFF78EFFFFF7A6FBE74C206830
:106F7000002800F09882E64D7103B0FBF5F0B1FBFC
:106F8000F0F000EE100AB8EE400ABCEEC00A10EEB7
:106F9000101A3F2988BF3F218C20FFF773FF20681C
:106FA0004FF40041B0FBF5F0B1FBF0F000EE100A39
:106FB000B8EE400ABCEEC00A10EE101A3F2988BF96
:106FC0003F21D220FFF75EFFD24D4FF00108691E2E
:106FD000287801280CBF40460020012291F802C009
:106FE0000023032411F10101BCF1000F11F8027F0D
:106FF00018BF08FA02FC604491F801C0C0B2002F2B
:107000001CBF571C08FA07F73B44921CDBB2641EF6
:10701000EAD1E9791844C0B2012914BF00218021C6
:107020000844DFF8F4A2C7B243F60959DAF80000C1
:10703000400190FBF9F15C20FFF724FFDAF804002F
:10704000400190FBF9F15D20FFF71CFFDAF8080022
:10705000400190FBF9F15E20FFF714FFDAF80C0015
:10706000400190FBF9F15F20FFF70CFFDAF8100008
:10707000400190FBF9F16020FFF704FFDAF81400FB
:10708000400190FBF9F16120FFF7FCFEDAF81800EF
:10709000400190FBF9F16220FFF7F4FEDAF81C00E2
:1070A000400190FBF9F16320FFF7ECFEAAF1140414
:1070B000DFF86882207801280CBF98F800100021C2
:1070C0006820FFF7DFFE607801280CBF98F80110F8
:1070D00000216920FFF7D6FEA07801280CBF98F8A0
:1070E000021000216A20FFF7CDFEE07801280CBFD6
:1070F00098F8031000216B20FFF7C4FE20790128C7
:107100000CBF98F8041000216C20FFF7BBFE6079DB
:1071100001280CBF98F8051000216D20FFF7B2FE82
:10712000A07901280CBF98F8061000216E20FFF707
:10713000A9FEE07901280CBF98F8071000216F2004
:10714000FFF7A0FE60219720FFF79CFE0121102091
:10715000FFF798FEDAF82000400190FBF9F1642077
:10716000FFF790FE207ADFF8B88101287ED0002159
:107170000F20FFF787FE00BFDAF82400400190FBE4
:10718000F9F16520FFF77EFE98F80000411EE62029
:10719000FFF778FE98F80000411EF420FFF772FE1A
:1071A00098F80000C0F10800C200D8E90401F9F71E
:1071B0001FF989460146ED20FFF764FE4946EE209F
:1071C000FFF760FE607A01287DD000211120FFF7D3
:1071D00059FEA0200121FFF755FEA2200021FFF754
:1071E00051FE00210920FFF74DFEA2200121FFF7EB
:1071F00049FEA1200121FFF745FEA3200021FFF752
:1072000041FE00210920FFF73DFEA3200121FFF7E9
:1072100039FE0121A020FFF735FE0121A120FFF753
:1072200031FE00219D20FFF72DFE00219E20FFF75B
:1072300029FE00219F20FFF725FE00215B20FFF79C
:1072400021FE0021A020FFF71DFE0021A120FFF755
:1072500019FE20214FF49770FFF714FE69464FF492
:107260008F70FFF7A3FD0098C0B200E003E0042890
:1072700040F019817AE0297AD920FFF703FE98F8C7
:10728000020001280ED0022807D0032840F00B810D
:107290000021D820FFF7F6FD08E00121D820FFF7F4
:1072A000F1FD03E00221D820FFF7ECFD98F8030080
:1072B00010281DD008DC02280BD004280ED0082886
:1072C00011D000F0F0B83BE0202816D0402829D09B
:1072D000E9E00721DE20FFF7D5FD27E00821DE20C9
:1072E000FFF7D0FD22E00921DE20FFF7CBFD1DE0F6
:1072F0000A21DE20FFF7C6FD18E00B21DE20FFF794
:10730000C1FD13E040160020300C00204802002090
:1073100040420F004A0C0020540C0020580200206C
:10732000300200200C21DE20FFF7ACFD98F804109D
:10733000DD20FFF7A7FD01210F20FFF7A3FD1BE7CD
:10734000697AEB20FFF79EFD5D49D8F80C00B1FB90
:10735000F0F1EC20FFF796FD98F80510E220FFF71A
:1073600091FD01211120FFF78DFD32E7202140F230
:107370002D10FFF787FD694640F21D10FFF716FD3F
:107380000098C0B201287DD1642003F005FB694656
:107390005020FFF70BFD0098102873D1494C0025B1
:1073A00094F85000002825DD10215B20FFF76AFDCE
:1073B000304603F0F1FA05EB8500204481784278ED
:1073C0000901C07801EB82110844C1B25B20FFF7CC
:1073D00059FD304603F0E0FA69465020FFF7E6FC1D
:1073E000009905F1300081425DD194F850006D1C88
:1073F000A842D9DCC0B2102814D210215B20FFF7BC
:1074000041FD304603F0C8FA11215B20FFF73AFD39
:10741000304603F0C1FA69465020FFF7C7FC0098D8
:10742000302840D110215B20FFF72CFD304603F0BF
:10743000B3FA03215B20FFF725FD304603F0ACFAD9
:1074400069465020FFF7B2FC009833282BD1102159
:107450005B20FFF717FD304603F09EFA00215B200A
:10746000FFF710FD304603F097FA69465020FFF70A
:107470009DFC0098302816D110215B20FFF702FDFB
:10748000304600E00FE003F087FA39465B20FFF753
:10749000F9FC304603F080FA69465020FFF786FC7D
:1074A0000098402803D04FF0FF30BDE8F88F00214E
:1074B0004FF49E70FFF7E6FC0020BDE8F88F000057
:1074C0000048E8016002002070B504464FF41771CF
:1074D000F9F7A8FB0021C4F85C12C4F86012C4F8E4
:1074E0006412C4F86812C4F86C12C4F87012C4F8BC
:1074F0007412C4F87812C4F87C12C4F88012C4F86C
:107500008412C4F88812C4F88C12C4F89012C4F81B
:107510009412C4F898120125C4F87459C4F860197B
:10752000D4F8780904F516620128D4F880090168B6
:107530004B6813D004F517719847C4F8745900BF0D
:10754000D4F874090028FBD1C4F8745904F52770E5
:10755000BDE8704040F2C461F9F764BB214698472A
:10756000F4E7000010B5044690F89E0294F89D12CE
:10757000042202EB0121084482B2D4F88009016898
:107580008B6804F52771984794F87C09012818BF87
:1075900010BDC82003F0F2F9BFF34F8F0548016812
:1075A000054A01F4E06111430160BFF34F8F00BF52
:1075B000FDE700000CED00E00400FA0510B5D0F87E
:1075C0008009016809688847BDE810404FF47A7067
:1075D00003F0D4B9A1F161001A2810D2DFE800F05D
:1075E0000D0D0D0D0F0D0F0D0D0D0F0D0D0D0F0DC3
:1075F0000D0D0D0D0D0F0D0D0D0D0120704700200F
:10760000704700002DE9F047044600202178ADF5D1
:10761000AD6D002909BF00208DF810110DF5AD6D7D
:10762000BDE8F08761391A2930D2DFE801F00D0D8D
:107630000D0D2F0D2F0D0D0D2F0D0D0D2F0D0D0DF2
:107640000D0D0D2F0D0D0D0D9DF8101161391A291D
:1076500080F0E485DFE811F0CF021703A6031204DF
:10766000E2055004E205E00320054205E20552056B
:10767000C005D005E2055B01FA0428006F00BE00DA
:107680000D01E205A901F2013B02870200206B21F6
:1076900084F89C1284F89D0284F89E0284F89F026C
:1076A0000DF5AD6DBDE8F08760788DF81101A37818
:1076B0004FF0FF368DF8123106EB0020E1781D18EF
:1076C000002D19DDE01C0DF2131213F0010F04D18F
:1076D00010F8013F8DF81431521C90F801C06B1066
:1076E0000AD000BF10F8025F82F801C090F801C014
:1076F00002F8025F5B1EF5D19DF811219DF8120181
:1077000006EB0222801804D4221844AB18441279E4
:107710000271FE4801F012FC722184F89C120021D3
:1077200084F89D12012184F89E1284F89F1284F837
:10773000A00200F07EB960788DF81101A3784FF0B7
:10774000FF368DF8123106EB0020E1781D18002D70
:1077500018DDE01C0DF2131213F0010F04D110F824
:10776000013F8DF81431521C90F801C06B1009D004
:1077700010F8025F82F801C090F801C002F8025FC1
:107780005B1EF5D19DF811219DF8120106EB022236
:10779000801804D4221844AB1844127902719DF861
:1077A00015019DF8142100EB0223732084F89C023C
:1077B0009DF8140184F89D029DF8150184F89E023D
:1077C000012084F89F0204F52872D04801F014FAD1
:1077D00000F02FB960788DF81101A3784FF0FF36D3
:1077E0008DF8123106EB0020E1781D18002D19DD0F
:1077F000E21C0DF2131013F0010F04D112F8013F37
:107800008DF81431401C92F801C06B100AD000BFF3
:1078100012F8025F80F801C092F801C000F8025F20
:107820005B1EF5D19DF811219DF8120106EB022295
:10783000801804D4221844AB1844127902719DF8C0
:1078400015019DF8142100EB0223742084F89C029A
:107850009DF8140184F89D029DF8150184F89E029C
:10786000012084F89F0204F52872A84801F0FAF973
:10787000DFE060788DF81101A3784FF0FF368DF8C6
:10788000123106EB0020E1781D18002D18DDE01CF8
:107890000DF2131213F0010F04D110F8013F8DF80F
:1078A0001431521C90F801C06B1009D010F8025F1F
:1078B00082F801C090F801C002F8025F5B1EF5D1AA
:1078C0009DF811219DF8120106EB0222801804D4C4
:1078D000221844AB1844127902719DF815019DF8E5
:1078E000142100EB0223752084F89C029DF81401FA
:1078F00084F89D029DF8150184F89E02012084F809
:107900009F0204F52872814801F04CF991E06078FB
:107910008DF81101A3784FF0FF368DF8123106EB88
:107920000020E1781D18002D18DDE01C0DF2131267
:1079300013F0010F04D110F8013F8DF81431521CDF
:1079400090F801C06B1009D010F8025F82F801C0F6
:1079500090F801C002F8025F5B1EF5D19DF811217D
:107960009DF8120106EB0222801804D4221844ABC1
:107970001844127902719DF815019DF8142100EB4D
:107980000223702084F89C029DF8140184F89D0263
:107990009DF8150184F89E02012084F89F0204F5E9
:1079A00028725A4801F0B8F843E060788DF8110168
:1079B000A3784FF0FF368DF8123106EB0020E17806
:1079C0001D18002D18DDE01C0DF2131213F0010F2D
:1079D00004D110F8013F8DF81431521C90F801C009
:1079E0006B1009D010F8025F82F801C090F801C056
:1079F00002F8025F5B1EF5D19DF811219DF812017E
:107A000006EB0222801804D4221844AB18441279E1
:107A100002719DF814213D4801F0CAFA772084F8DC
:107A20009C02002084F89D0284F89E02012084F8C4
:107A30009F020DF5AD6D0120BDE8F08760788DF8EF
:107A4000110194F802C04FF0FF370CEB00238DF8C2
:107A500012C107EB0020E1780CEB0006002E18DDC8
:107A6000E01C0DF213121CF0010F04D110F801CF2D
:107A70008DF814C1521C45785FEA660C09D000BF2E
:107A800010F8026F5570457802F8026FBCF1010CD6
:107A9000F6D19DF811219DF8120107EB0222801802
:107AA00005D422180DF5887C60441279027145AA2C
:107AB000164801F05DF9782084F89C02002084F8D3
:107AC0009D0284F89E02012084F89F02B1E760784D
:107AD0008DF8110194F802C04FF0FF370CEB002332
:107AE0008DF812C107EB0020E1780CEB0006002EA8
:107AF0001BDDE01C0DF213121CF0010F04D110F875
:107B000001CF8DF814C1521C457801E040160020C9
:107B10005FEA660C09D000BF10F8026F5570457817
:107B200002F8026FBCF1010CF6D19DF811219DF80D
:107B3000120107EB0222801805D422180DF5887C6B
:107B400060441279027145AAFE4801F045F9792096
:107B500084F89C02002084F89D0284F89E02012093
:107B600084F89F0265E760788DF8110194F802C0EF
:107B70004FF0FF370CEB00238DF812C107EB00200C
:107B8000E1780CEB0006002E17DDE01C0DF213125D
:107B90001CF0010F04D110F801CF8DF814C1521C54
:107BA00045785FEA660C08D010F8026F557045788A
:107BB00002F8026FBCF1010CF6D19DF811219DF87D
:107BC000120107EB0222801805D422180DF5887CDB
:107BD00060441279027145AADA4801F0A1F87A20CE
:107BE00084F89C02002084F89D0284F89E02012003
:107BF00084F89F021DE760788DF8110194F802C0A7
:107C00004FF0FF370CEB00238DF812C107EB00207B
:107C1000E1780CEB0006002E17DDE01C0DF21312CC
:107C20001CF0010F04D110F801CF8DF814C1521CC3
:107C300045785FEA660C08D010F8026F55704578F9
:107C400002F8026FBCF1010CF6D19DF811219DF8EC
:107C5000120107EB0222801805D422180DF5887C4A
:107C600060441279027145AAB64801F013F8612008
:107C700084F89C02002084F89D0284F89E02012072
:107C800084F89F02D5E6607800268DF81101A2786D
:107C9000771E07EB002002EB000C4FF49679354677
:107CA0008DF81221BCF1000F16DDE01C0DF213114E
:107CB00012F0010F04D110F8012F8DF81421491C86
:107CC00043785FEA6C0207D010F802CF4B7043781C
:107CD00001F802CF521EF7D19DF811119DF8120143
:107CE00007EB0121401804D4211844AA1044097953
:107CF00001719DF814019449FEF708F9B0F1000CE8
:107D00004FF0620084F89C024FF0010101EBEC702F
:107D100084F89F0284F8A0C24FF00007C4BFDFF8C8
:107D20002882A9F5807236DDC7EB071000EB8000D2
:107D300008EB8001488D8318002B28DD002350407C
:107D400010F0010005D005EB04090B7889F8A13289
:107D50000123B1F82A909144814515DD05EB030A12
:107D600011F80390A2445B1C8AF8A19205EB030A68
:107D7000A24411F803908AF8A192B1F82A90801CCD
:107D800091445B1C8145E9DC488D304486187F1C9A
:107D90003546BC45C8DC701C010A84F89D1284F885
:107DA0009E0246E660788DF81101A2788DF81221C6
:107DB00094F803C012EB002019D0E01C0DF28F31B3
:107DC00012F0010F03D010F8012F01F8012F9DF8D8
:107DD00012219DF8113102EB0322520807D043789B
:107DE0004B7010F8023F01F8023F521EF7D1DDE957
:107DF000E701CDE90001DDE9E4126046E69BFEF70C
:107E0000F1FB632184F89C12002184F89D1284F810
:107E10009E1200286FD017E160788DF81101A278CA
:107E20008DF8122112EB002019D0E01C0DF2C74191
:107E300012F0010F03D010F8012F01F8012F9DF867
:107E400012219DF8113102EB0322520807D043782A
:107E50004B7010F8023F01F8023F521EF7D10DF5AA
:107E60009960FEF7F3FB682184F89C12002184F8E6
:107E70009D1284F89E1200283DD0E5E060788DF8D0
:107E80001101A2788DF8122194F803C012EB0020A2
:107E900019D0E01C0DF26F3112F0010F03D010F871
:107EA000012F01F8012F9DF812219DF8113102EBED
:107EB0000322520807D043784B7010F8023F01F8B4
:107EC000023F521EF7D1DEAF97E86F008DE86F00DA
:107ED000DDE9DC236046FEF771FA642184F89C1228
:107EE000002184F89D1284F89E12002803D0ABE094
:107EF00084F89F029DE5A5E00DF5AA6000F09BFCCB
:107F000060788DF81101A2788DF8122112EB002013
:107F10001ED0E01C0DF2A73112F0010F03D010F8B3
:107F2000012F01F8012F9DF812219DF8113102EB6C
:107F3000032252080CD043784B7010F8023F01F82E
:107F4000023F03E0401600202C170020521EF2D101
:107F5000B94DB5F90000B0F1FF3F04D13422B7A10B
:107F6000C6A001F041FFA888E96800040860C94D77
:107F700001266E712E714FF48872EEA96846F8F7EB
:107F80001FFEEAAF97E80F00FEF7C4FC0DF5AC61E9
:107F9000BD20FEF70BFFDDF8600501281BD00DF5B5
:107FA000AA6000F014FC0DF5AA6000F01EFCBA4EA9
:107FB000287938B10DF5AA6000F0D0FB10EE100A58
:107FC000B042F5DB0DF5AA6000F0E8FB95F8200063
:107FD00001281BD10AE0662084F89C02002084F866
:107FE0009D0284F89E0284F89F6222E50DF24C50B7
:107FF000FEF7D4F905F1080000F007FCDDF84C1598
:10800000401A3C30E861002085F82000A14801F0CA
:108010000DF8894DB5F90000B0F1FF3F04D13422CD
:1080200086A196A001F0E0FEE96868680860FEF7A6
:108030006FFF662184F89C12002184F89D1284F859
:108040009E1208B9012053E7002051E7DBA8FEF794
:10805000A5F901008F48DB9A806910444FF0710246
:10806000DB9084F89C224FF0000284F89D224FF0B0
:10807000040284F89E220CBF0121002184F89F1283
:10808000010E84F8A012010C84F8A112010A84F8F0
:10809000A21284F8A302CCE461788DF81111A278C1
:1080A0008DF8122102EB0122002AC8BF0DF26453A1
:1080B00005DD211809791954401C8242F9DCDDF8EC
:1080C0006405FEF7BDFA692184F89C12002184F84A
:1080D0009D1284F89E120028B6D1B3E76179207909
:1080E000FEF78CFB6A2084F89C02002084F89D0235
:1080F00084F89E02012084F89F029AE460788DF84B
:108100001101A2784FF0FF3505EB002C02EB0C00BB
:108110008DF81221002817DDE01C0DF2131112F06A
:10812000010F04D110F8013F8DF81431491C437838
:108130006244521008D000BF10F802CF4B70437851
:1081400001F802CF521EF7D19DF811119DF81201CE
:1081500005EB0121401804D4211844AA10440979E0
:108160000171E0792179A27900EB0160617909045C
:1081700001EB022101446C2084F89C02002084F869
:108180009D02082284F89E22A1F18572921F08BFE9
:10819000012084F89F024148007884F8A0024048FA
:1081A000007884F8A1023F48007884F8A2023E4893
:1081B000007884F8A3023D48007884F8A4023C4883
:1081C000007884F8A5023B48007884F8A6023A4873
:1081D000007884F8A7022CE4FEF7D2F86D2084F82A
:1081E0009C02002084F89D0284F89E02012084F8FD
:1081F0009F0284F87C091CE410213048FDF700FE42
:108200006E2084F89C02002084F89D0284F89E026F
:10821000012084F89F0284F87C090AE46B2084F82A
:108220009C02002084F89D0284F89E0284F89F023C
:108230000DF5AD6DBDE8F0871C1700206D6265641B
:108240002D6465762F746172676574732F68616C35
:108250002F5441524745545F53544D2F5441524778
:1082600045545F53544D333246342F6770696F5F06
:108270006F626A6563742E68000000006F626A2D89
:108280003E70696E20213D202850696E4E616D65FB
:10829000294E43004016002000002041187AFF1F9D
:1082A000197AFF1F1A7AFF1F1B7AFF1F107AFF1F10
:1082B000117AFF1F127AFF1F137AFF1F00100108A7
:1082C00070B50446002084F87C0915460E46D82077
:1082D00000F096FF78B131462A46002300F0C2FA3A
:1082E000084940F8BC1B683140F804193C3940F893
:1082F0001C1B4C310160C4F880090120C4F87809C6
:10830000204670BD58BD000870B504460068416A3B
:1083100020468847206801220021036920469847AB
:108320000546B0F1FF3F206811D002220369002109
:1083300020469847064620680022294603692046C1
:1083400098472068816A20468847304670BD816A18
:10835000204688474FF0FF3070BD70477047483067
:1083600001F030BF10B50C46483002F0CDF8204681
:1083700010BD00EB011000F19401D0F8A020002AFC
:1083800008BF70478868104770B50446483002F04F
:108390000DF8236C054600F47C52002B18BF002A10
:1083A00003D004F13401E06B9847236B05F0FC0225
:1083B000002B14BF002A70BD04F12401E06ABDE85F
:1083C0007040184770B5044600680D4601682046A5
:1083D0008847294604F1480001F0F0FEC4F8B45083
:1083E000206841682046BDE87040084770477047E4
:1083F00070B50446006801682046884704F14800CB
:1084000002F094F8054620684168204688472846CF
:1084100070BD000070B50E46044620491E48154642
:108420002060D1E902230021A260E3601C4A22619E
:10843000A161646104F10801E1611A492162BFF39D
:108440006F8FBFF34F8F00216162216361632164ED
:1084500084F8441084F845104C2104F14800F8F7E2
:10846000E1FB02231022104904F1940000F014FFF4
:10847000A0F194044FF41650C4F8B4002A463146D3
:1084800004F1480001F0AEFE2246084904F148001C
:1084900001F080FF204670BD18BE0008CCAC00087B
:1084A0009FE8078049AA0008893000087383000804
:1084B000002908BF704701290AD0022918BF704758
:1084C00000F13401026C002A08BF70478868104729
:1084D000026B00F12401002AF8D1704770B50D46F7
:1084E000044601F0C9F8E868002804F134000DD012
:1084F000A9688160D5E90012C0E90012E968C1608D
:1085000001220221203801F053FB08E00021016024
:10851000C1600A46022104F1140001F049FBBDE8E4
:10852000704001F0FDB8000070B504460D4800220F
:10853000C4E90002A260E26022616261A261E261BC
:10854000226262622263626322640D462346064A07
:1085500004F1140001F08AFA2946201D01F0B5F952
:10856000204670BD30BE0008B184000810B5044636
:108570000348206004F1140001F052FA204610BDB7
:1085800030BE00080021F8F725BA0000074801684E
:10859000002904BF011D0160001D814208BF704712
:1085A00056220349034801F01FBC000018020020B6
:1085B00074BF000860BF000870B5044600680E462E
:1085C00041682046884720684168204688470F4D0B
:1085D0002868A0420AD0D4E90A120023201D01F025
:1085E000B1FF201D216B01F0E1FF2C602068816844
:1085F000204688473146201D02F0FEF805462068D7
:10860000816820468847284670BD0000140200207B
:1086100070B5044600680D461646416820468847F6
:10862000C4E90A560F4D00202860206841682046A2
:1086300088472868A0420AD0D4E90A120023201DE6
:1086400001F080FF201D216B01F0B0FF2C6020683D
:10865000816820468847206881682046BDE87040D0
:10866000084700001402002007480168002904BFE1
:10867000011D0160001D814208BF70475622034959
:10868000034801F0B1BB00001802002074BF0008CD
:1086900060BF000870B5044600680D46416820467A
:1086A000884725630F4D00202860206841682046D8
:1086B00088472868A0420AD0D4E90A120023201D66
:1086C00001F040FF201D216B01F070FF2C6020683D
:1086D000816820468847206881682046BDE8704050
:1086E000084700001402002038B504461848DDF899
:1086F00010C0206000206060A060E06020616061C8
:10870000A061E06108252062C4E90905E062114822
:108710002063201DCDF800C001F0A4FF206841684F
:10872000204688470C4D2868A0420AD0D4E90A1296
:108730000023201D01F006FF201D216B01F036FFF4
:108740002C602068816820468847204638BD00009C
:1087500040BE000840420F001402002070B50446DD
:1087600000F08AFF00F088FF2068002520B1E06853
:1087700002F081F86168451A00F0D2FFA0682C1859
:1087800000F0CEFF00EE104A9FED031AF8EEC00A8B
:1087900080EE810A70BD00000024744970B5044663
:1087A00000F06AFF00F068FF2068002520B1E06853
:1087B00002F061F86168451A00F0B2FFA068284431
:1087C000A06000202060BDE8704000F0A9BF10B597
:1087D000044600F051FFE06802F04DF860600020B0
:1087E000A060BDE8104000F09BBF10B5044600F04B
:1087F00043FF206828B9E06802F03DF8606001207E
:108800002060BDE8104000F08BBF70B5044600F05A
:1088100033FF00F031FF2068002520B1E06802F04E
:108820002AF86168451A00F07BFFA0682C1800F058
:1088300077FF204670BD70B5002505604560044691
:10884000856000F0DBFFE06000F016FFE06802F0FA
:1088500012F8C4E9010500F063FF204670BD7047BF
:108860007047000010B51C46FFF7D4FD2146B83014
:1088700000F078F8044940F8B81D5C31C0F8BC102D
:108880003C39C0F8B81010BD5CBE0008002070472D
:1088900070B504460068416A204688476069F8F769
:1088A0000CF8606900F035F905462068816A2046B9
:1088B0008847284670BD70B5044600680D46416A79
:1088C000204688476069F7F7F8FF2846616900F09D
:1088D00087FF05462068816A20468847284670BD84
:1088E0002DE9F041054600680F460C468E18416A96
:1088F00028468847B4420AD02868026B2846904729
:10890000B0F1FF3F03D004F8010BB442F4D1286862
:10891000816A28468847E01BBDE8F0810020704747
:10892000002070472DE9F041054600680F460C46CF
:108930008E18416A28468847B4420AD0286814F83D
:10894000011BC26A28469047B0F1FF3F18BFB442EE
:10895000F4D12868816A28468847E01BBDE8F08189
:108960000020704710B584B000F074F804460A483F
:1089700020603C30606000206061224607A16846AC
:10898000F7F75CFD06A16846F7F7FDFF6061FFF7AA
:10899000F9FD04B0204610BDC8BE00083A2570009D
:1089A000772B0000007B704770B506460D461548D2
:1089B00002F02AF814480468F4B1A068C8B12A4645
:1089C0003146F8F76DF8A0B9A068F8F74AF8A84260
:1089D0000FD10C480168002904BF011D0160001D72
:1089E000814204D056220949094801F0FDF9204688
:1089F00070BD6468002CE0D1024802F005F8002048
:108A000070BD0000F4010020F001002074BF0008D8
:108A100060BF000870B504460B480026A160C4E999
:108A200000060D462273094801F0EEFF002D08BF35
:108A3000666003D00648016861600460034801F085
:108A4000E3FF204670BD000014BF0008F4010020C1
:108A5000F001002010B5064A40F8042B0022FFF771
:108A6000D9FF044940F8041D3431416010BD0000B5
:108A7000E4BD000824BF000810B50446406828B1D2
:108A8000FFF790FF012804BF606810BD002010BDF3
:108A900010B50446406810B1FFF784FF08B100200C
:108AA00010BD6068002818BF001F10BD4068002876
:108AB00018BF0120704710B54068002808BF10BDDE
:108AC000FFF770FF00280CBF0120002010BD0068D8
:108AD000704710B5044600202060606008782F2899
:108AE0000DD1487858B14B1C0021236022681078C2
:108AF0002F2806D038B1501C491C2060F6E72046CC
:108B000010BD501C20601846FFF74EFF60602046E5
:108B100010BD00F059BE00002DE9F0471E46174673
:108B2000894604464FF0000872B600F12405B0F9FA
:108B30002400B0F1FF3F05D11949342201F1400072
:108B400001F052F9A888E968000408600A2001F0E1
:108B500023FF09F07F0104F14400FFF72DFD0025FC
:108B6000002E08DD002104F14400FFF725FD7855B3
:108B70006D1CAE42F6DC012001F00EFF34F9240F2B
:108B8000B0F1FF3F05D10649342201F1400001F068
:108B90002BF9E1686068086062B64046BDE8F0877E
:108BA0007C9000082DE9F0411E1E174604464FF048
:108BB000000872B6454608DD002104F14400FFF7C5
:108BC000FBFC78556D1CAE42F6DC012001F0E4FEA2
:108BD00034F9240FB0F1FF3F05D10649342201F1E9
:108BE000400001F001F9E1686068086062B6404643
:108BF000BDE8F0817C9000082DE9F0471E4617463D
:108C0000894604464FF0000872B600F12405B0F919
:108C10002400B0F1FF3F05D11149342201F1400099
:108C200001F0E2F8A888E96800040860012001F07A
:108C3000B3FE09F07F0104F14400FFF7BDFC0025FD
:108C4000002E08DD002104F14400FFF7B5FC785543
:108C50006D1CAE42F6DC62B64046BDE8F08700000F
:108C60007C9000082DE9F0411D1E164607464FF086
:108C7000000872B6444608DD002107F14400FFF702
:108C80009BFC3055641CA542F6DC62B64046BDE84C
:108C9000F08100002DE9F0471F46904689460446C2
:108CA000002572B600F12406B0F92400B0F1FF3FB0
:108CB00005D11A49342201F1400001F095F8B0883D
:108CC000F16800040860012001F066FE09F07F00F1
:108CD00040F0800104F14400FFF76EFC002F08DD36
:108CE00018F8051004F14400FFF766FC6D1CAF4254
:108CF000F6DC012001F050FE34F9240FB0F1FF3F03
:108D000005D10649342201F1400001F06DF8E16817
:108D10006068086062B6BDE8F08700007C900008DB
:108D20002DE9F0411E1E174604464FF0000572B6AD
:108D300007DD795D04F14400FFF73EFC6D1CAE4297
:108D4000F7DC012001F028FE34F9240FB0F1FF3FD9
:108D500005D10649342201F1400001F045F8E168EF
:108D60006068086062B6BDE8F08100007C90000891
:108D70002DE9F0471F46904689460446002572B605
:108D800000F12406B0F92400B0F1FF3F05D11149EC
:108D9000342201F1400001F027F8B088F1680004A6
:108DA0000860012001F0F8FD09F07F0040F080012B
:108DB00004F14400FFF700FC002F08DD18F805104F
:108DC00004F14400FFF7F8FB6D1CAF42F6DC62B61D
:108DD000BDE8F0877C9000082DE9F0411D1E164685
:108DE00007464FF0000472B607DD315D07F144001D
:108DF000FFF7E2FB641CA542F7DC62B6BDE8F08138
:108E0000F0B5444D044685B0B5F90000B0F1FF3F20
:108E100005D14149342201F1400000F0E5FFE96845
:108E2000686808603D4DB5F90000B0F1FF3F05D11D
:108E30003949342201F1400000F0D6FFE968686842
:108E40000860B4F9340004F13405B0F1FF3F05D1F6
:108E50003149342201F1400000F0C6FFE96868683A
:108E600008600A2001F098FDB4F9340004F13405DB
:108E7000B0F1FF3F05D12849342201F1400000F054
:108E8000B3FFA888E968000408600A2001F084FDA7
:108E9000B4F9240004F12405B0F1FF3F05D11E49C7
:108EA000342201F1400000F09FFFE9686868086023
:108EB0000A2001F063FD0022082104F14400FFF7BD
:108EC000A7FB174904F14400FFF7E4FB154804F140
:108ED0007807D0E9005600F0CFFB1348CDE90056E3
:108EE000CDE9024069463846FFF7F8FA00F018FC71
:108EF000012084F8200000206071A06104F10800C6
:108F0000FFF765FC04F10800FFF76FFC05B00120D6
:108F1000F0BD0000FC1600207C9000081C1700200B
:108F200000127A003CBC000835AA000872B64179EC
:108F3000012904BF0021017162B6704770B50E4669
:108F4000044672B600F12405B0F92400B0F1FF3FE9
:108F500005D11649342201F1400000F045FFA888F0
:108F6000E96800040860012001F016FD06F07F01A9
:108F700004F14400FFF720FB002104F14400FFF757
:108F80001BFBC5B2012001F007FD34F9240FB0F13D
:108F9000FF3F05D10549342201F1400000F024FFD4
:108FA000E1686068086062B6284670BD7C90000881
:108FB0002DE9F04117460E46044672B600F124052D
:108FC000B0F92400B0F1FF3F05D11749342201F177
:108FD000400000F009FFA888E9680004086001204B
:108FE00001F0DAFC06F07F0040F0800104F144005B
:108FF000FFF7E2FA394604F14400FFF7DDFA0120F9
:1090000001F0CAFC34F9240FB0F1FF3F05D1064945
:10901000342201F1400000F0E7FEE168606808607A
:1090200062B6BDE8F08100007C90000870B504468F
:1090300000F13405B0F93400B0F1FF3F04D134221F
:109040000EA11EA000F0D0FEE968686808600A2042
:1090500001F0A2FC34F9340FB0F1FF3F04D1342207
:1090600006A116A000F0C0FEA088E1680004086018
:10907000BDE870400A2001F08FBC00006D6265649D
:109080002D6465762F746172676574732F68616CE7
:109090002F5441524745545F53544D2F544152472A
:1090A00045545F53544D333246342F6770696F5FB8
:1090B0006F626A6563742E68000000006F626A2D3B
:1090C0003E70696E20213D202850696E4E616D65AD
:1090D000294E43002DE9F84F0E46DDE90A5A16499C
:1090E000DDF830B09846914640F8081BFFF7A3FB27
:1090F000A0F10804002740F81C7F314647608760D4
:10910000C76000F0F7FB6763A763E76304F134000F
:109110005946276400F0EEFB781E00902B4642462D
:10912000494604F14400FFF7DFFA51463430FFF7B7
:10913000FBF97838BDE8F88F4CBD000810B503493D
:1091400040F8781BFFF712FA783810BD4CBD0008C4
:109150007047B838FFF703B9B838FFF703B970475D
:109160004FF4E131D438FFF72DB92DE9F0419046A5
:10917000A0F1D4050C4600262846FFF739F901284E
:1091800006D105F1B800FFF783FBA055701C86B22D
:10919000042EF1D3A0786178002600EB01200704AB
:1091A0003F0C0ED02846FFF723F9012807D105F11F
:1091B000B800FFF76DFBA1190871701C86B2BE42A2
:1091C000F0D3381DC8F80000BDE8F0812DE9F0416A
:1091D000A0F1D4070E46144612F03F0F04BF501CF6
:1091E00084B20025002CD8BFBDE8F081715D07F185
:1091F000B800FFF760FB6D1CAC42F7DCBDE8F08106
:1092000010B5F7F79FF8040004BF02A000F0C2FAFF
:10921000204610BD4F70657261746F72206E657765
:10922000206F7574206F66206D656D6F72790D0A01
:109230000000000003B401984100009850EAC120EA
:1092400018BF04204A0D18BF40F0010040F2FF7221
:10925000B2EB515F08BF40F00200012808BF0520B3
:1092600002B070472DE9F0410A4D0E4607462C68C2
:109270002868B0F1006F08D12146AC064FF4CA72DD
:109280002046F7F79DFC2046286004EB8700066423
:10929000BDE8F08108ED00E02DE9F0411C461746DD
:1092A0000E00804607D0054602E02846B0473D4400
:1092B0002046641EF9D24046BDE8F0810020F8F750
:1092C00064BB00000A2209210148FEF7F9BF000033
:1092D000BC0C002010B584B005200090032214219E
:1092E000CDE901120623072204211148FFF7F2FEFF
:1092F000104A1149F7F79EFB104800241021046022
:1093000044608460C46000F0F5FA0D4821460460B2
:1093100044608460C46000F0EDFA0A4812210460E1
:1093200044608460C46004B0BDE8104000F0E2BA5C
:1093300040160020000000083D910008FC160020A7
:109340000C1700201C17002002486A4620F0070076
:10935000704700000F2B002030380A2801D201206E
:1093600070470020704700000328BCBF00207047F2
:109370000749002201EB800151F80C0C41F80C2C3C
:10938000002804BF4FF0FF30704701684968084764
:10939000380800200328BCBF00207047064901EBB5
:1093A000800050F80C0C002804BF4FF0FF307047CD
:1093B0000168896908470000380800200328BCBFFD
:1093C00001207047064901EB800050F80C0C002882
:1093D00004BF4FF0FF3070470168C96808470000BC
:1093E000380800202DE9F0430E4683B081466149DC
:1093F000F7F740FC604C10B360494846F7F73AFC79
:1094000040B35F494846F7F735FC70B35D4C2068C0
:10941000002804BF201D2060251DA84204D056222C
:1094200059495A4800F0E0FC2168594F002400BF18
:1094300057F8240028B3641C102CF9D323E02068CB
:1094400020B903220221534800F0CCFE03B00020D3
:10945000BDE8F083206820B9032202214D4800F0C6
:10946000C1FE03B00120BDE8F083FFE7206820B90A
:1094700003220221474800F0B5FE03B00220BDE8F8
:10948000F083102C11D33F48002904BF011D016057
:109490000068A84204D056223B493C4800F0A4FC96
:1094A00003B04FF0FF30BDE8F0834FF0FF3047F8D6
:1094B00024003448002904BF011D01600068A8424F
:1094C00004D056223049314800F08EFC99F8000053
:1094D0004FF000083A2810D049466846FFF7F9FADD
:1094E0006846FFF7E3FA98B36846FFF7E4FA002806
:1094F000684609D0FFF7CCFA22E06A4626A1484622
:10950000F7F7FCF800981BE0FFF7B6FA00B316F087
:10951000020F18BF022522D016F00C0F18BF45F419
:10952000007516F0040F18BF45F4806506466846BE
:10953000FFF7CDFA014630682A46836830469847DF
:1095400000281FBF47F82400E01C03B0BDE8F083EB
:1095500047F8248003B04FF0FF30BDE8F08316F0E9
:10956000040F18BF0125D7D116F0080F14BF092525
:109570000025D1E7B4AC0008E0010020BBAC000836
:10958000C3AC00080C02002074BF000860BF0008D4
:1095900038080020380700203A25700070B51446BE
:1095A0000D4603280DDA0F48006820B90322022176
:1095B0000D4800F017FE0C4800F004FE2870012052
:1095C0000DE00A4901EB800050F80C0C002804BFA4
:1095D0004FF0FF3070BD01688B6829469847201A0C
:1095E00070BD0000E001002038070020380800208E
:1095F0000328BCBF00207047064A02EB800050F8E9
:109600000C0C002804BF4FF0FF307047026813694C
:10961000002218473808002070B514460E4603286B
:1096200013DA1248006820B903220221104800F022
:10963000D9FD0025002C06D9715D0D4800F064FFAE
:109640006D1CAC42F8D820460DE00A4901EB8000C1
:1096500050F80C0C002804BF4FF0FF3070BD0168BB
:109660000B6831469847201A70BD0000E0010020C9
:10967000380700203808002070B5EFF31080012172
:1096800021EA000080F0010572B60D4C60680028E8
:1096900008BF25706068B0F1FF3F04D1322209A1F4
:1096A00010A000F0A1FB606828B125B9362205A101
:1096B00016A000F099FB6068401C606070BD00005F
:1096C000FC0100206D6265642D6465762F636F6D0B
:1096D0006D6F6E2F6D6265645F637269746963613B
:1096E0006C2E6300696E746572727570745F656E5E
:1096F00061626C655F636F756E746572203C2055A6
:10970000494E5433325F4D4158000000696E746514
:109710007272757074735F64697361626C65640002
:1097200010B50E4C6068002808BF10BDEFF3108024
:10973000012121EA000090F0010F04D1472208A185
:109740000FA000F051FB6068401E60606068002858
:1097500006BF2078002810BD62B610BDFC010020B5
:109760006D6265642D6465762F636F6D6D6F6E2F0E
:109770006D6265645F637269746963616C2E630016
:10978000696E74657272757074735F646973616217
:109790006C6564000FB410B503A9029800F0CEFB0D
:1097A000012000F001F8000004460548F7F785F8AD
:1097B0000448F7F782F8002C18BF00F03FFBFEE7E3
:1097C000402A0020942A00200168002901DCF7F7D4
:1097D0002EBD491E016041684A1C426008787047EE
:1097E0008A68002A01DCF7F710BE521E8A604A68B8
:1097F000C0B2531C4B6010707047000000487047A7
:10980000ACAC000870B50446B0F900000D46B0F1EC
:10981000FF3F04D1462209A117A000F0E5FAB4F9F0
:109820000000012D04D0BDE87040002100F0B4BB61
:10983000BDE87040012100F0AFBB00006D626564BF
:109840002D6465762F746172676574732F68616C1F
:109850002F5441524745545F53544D2F5441524762
:1098600045545F53544D333246342F6770696F5FF0
:109870006170692E630000006F626A2D3E70696E30
:1098800020213D202850696E4E616D65294E4300B0
:1098900070B50C4605460180B1F1FF3F08BF70BDB1
:1098A000C4F30310FBF77EF806460021204600F0C3
:1098B00073FB04F00F00012101FA00F0686006F16B
:1098C0001000A8600830E86070BD70B5002605463D
:1098D0000C46FFF7DDFFB4F1FF3F08BF70BD00216C
:1098E0002846FFF78FFF31462846BDE8704000F05C
:1098F0009BB9000070B504460D460026FFF7C8FF6F
:10990000B5F1FF3F08BF70BDB4F90000B0F1FF3FF3
:1099100005D10A49342201F1400000F065FAA0881F
:10992000E1680004086001212046FFF76BFF314623
:109930002046BDE8704000F077B90000909900081B
:109940002DE9F04104460E4600271546FFF7A0FF1B
:10995000B6F1FF3F08BFBDE8F081B4F90000B0F1F7
:10996000FF3F04D134220AA119A000F03DFA002DD6
:1099700012BF6068A0880004E168086001212046E9
:10998000FFF740FF39462046BDE8F04100F04CB9F2
:109990006D6265642D6465762F746172676574739A
:1099A0002F68616C2F5441524745545F53544D2FDB
:1099B0005441524745545F53544D333246342F6718
:1099C00070696F5F6F626A6563742E6800000000E3
:1099D0006F626A2D3E70696E20213D202850696EAD
:1099E0004E616D65294E43000121002000F020B931
:1099F0000121084600F01CB90121022000F018B92D
:109A00000121032000F014B90121042000F010B955
:109A10000521084600F00CB90621084600F008B9F7
:109A200070B504464068104A00EB400101EB00109D
:109A30000C49012301EB8000217B002501F00F017F
:109A400052F8211002688B409A43026000EB8100BB
:109A500029464560C5614563B4F90C0000F09CFAE5
:109A6000A56070BD04030020A00100202DE9F84F7F
:109A70009A4693460F468046B1F1FF3F04BF4FF030
:109A8000FF30BDE8F88FC7F3031007F00F09B9F1F5
:109A9000100F5DD2DFE809F0080C1014181C1C1C14
:109AA0001C1C20202020202006242D4E002516E0FE
:109AB00007242C4E012512E008242B4E02250EE02F
:109AC00009242A4E03250AE00A24294E042506E02B
:109AD0001724284E052502E02824274E0625FAF7EC
:109AE00061FF00900721384600F056FA31462046C3
:109AF000FFF7B8FB04F01F00012202FA00F0610931
:109B0000890001F1E021C1F8000188F8004000203F
:109B1000C8E9015005EB4500184900EB051001EBC1
:109B200080001749A8F80C70036851F829108A4082
:109B30001A4300EB81010260C1F804A00098C1F84B
:109B40003490C8610F48C0F800B00020BDE8F88F1D
:109B50000DA0FFF71FFE4FF0FF30BDE8F88F0000AB
:109B6000E9990008F1990008F9990008019A00089C
:109B7000099A0008119A0008199A000804030020A5
:109B8000A00100209C010020496E746572727570FE
:109B900074496E206572726F723A2070696E206E21
:109BA0006F7420737570706F727465642E0A000094
:109BB00030B40B460C21012402254FF0000CB2B149
:109BC0000322012B02D0022B0BD01DE08168022959
:109BD00018BF032902D10821826015E006218460A4
:109BE00012E08168012918BF032914D1F3E7012B82
:109BF00002D0022B12D007E08268022A18BF032A83
:109C000009D000BFC0F808C0B0F90C0030BC6CF33C
:109C10001F1100F0C1B907218560F5E78268012AAC
:109C200018BF032AEED1D9E7B0F9000000F004BA5A
:109C30002DE9F0470E0000EB400101EB001019493F
:109C40004FF0000401EB800508BFBDE8F087012755
:109C5000DFF85480DFF85490296807FA04F00142D5
:109C60001AD005EB8400D8F8003090F83420C16990
:109C700007FA02F213420FD0C8F80020406858B12A
:109C80000969114204D1D9F800200221904703E06C
:109C9000D9F8002001219047641CB442DCD3BDE810
:109CA000F087000004030020143C01409C010020C8
:109CB00010B5144C016821600A6822F040020A6065
:109CC000016961608169E1610021A160C26862612E
:109CD000826822610722C4E90A124268E2602162B6
:109CE00040696162A0612046FAF7B6FB00281CBFFC
:109CF00005A0FFF74FFD2068016841F040010160B9
:109D000010BD00008407002043616E6E6F742069EF
:109D10006E697469616C697A65205350490000006E
:109D200010B5194A416802EB81140168216081680D
:109D30006160C168A1600169E16041692161016AF6
:109D4000A1610021E161E184A184E185A185B0F9EF
:109D50001A10B1F1FF3F04BF0820606107D0B0F9CD
:109D60001800B0F1FF3F0CBF04200C206061FAF72F
:109D700089FE2046FAF754FD002808BF10BD03A055
:109D8000BDE81040FFF706BD3805002043616E6E48
:109D90006F7420696E697469616C697A65205541D8
:109DA00052540A000D480178102905D1FF21FCF713
:109DB00027F80B4840688047FCF79AF80948FDF7F8
:109DC000FDFB0848FDF780FB0648FDF71BFC00285B
:109DD0001CBF0448FDF7C6FBF3E7000000100108B4
:109DE0000000FF1FBC0C002070B514460D4606464F
:109DF000FFF742FC23462A46314603A000F074F8E0
:109E0000BDE8704000F01AB86D626564206173733C
:109E10006572746174696F6E206661696C65643A1D
:109E20002025732C2066696C653A2025732C206CE4
:109E3000696E65202564200A0000000084B0FFF7E9
:109E40001BFC05216846FFF755FD00BFBDF900006A
:109E5000B0F1FF3F04D134220DA11DA0FFF7C4FFD4
:109E6000039901980860962000F088FDBDF9000074
:109E7000B0F1FF3F04D1342205A115A0FFF7B4FFD4
:109E80000198039900040860962000F077FDDDE753
:109E90006D6265642D6465762F7461726765747395
:109EA0002F68616C2F5441524745545F53544D2FD6
:109EB0005441524745545F53544D333246342F6713
:109EC00070696F5F6F626A6563742E6800000000DE
:109ED0006F626A2D3E70696E20213D202850696EA8
:109EE0004E616D65294E43000FB470B5A0B025AC2E
:109EF000249DFFF7C1FB224629466846F6F78CFAF7
:109F0000051E10DD0B48006820B9032202210A4813
:109F100000F068F900246E460748315D00F0F4FA5D
:109F2000641CAC42F8DBFFF7FBFB20B070BC5DF8B3
:109F300014FB0000E00100203807002070B5A0B03D
:109F40000C460546FFF798FB224629466846F6F779
:109F500063FA051E10DD0A48006820B903220221B9
:109F6000084800F03FF900246E460648315D00F0D5
:109F7000CBFA641CAC42F8DBFFF7D2FB20B070BD1B
:109F8000E001002038070020704710B5FAF77AFD8D
:109F9000BDE81040F9F7CEBAF0B585B00C460546DD
:109FA000B0F1FF3F04D181220FA11DA0FFF71CFFDC
:109FB00004F00F07C4F30216C5F30310C4F3C3146F
:109FC00005F00F05FAF7EEFC0121A94000911949AF
:109FD00051F82710CDE901160321CDE90314694694
:109FE000F9F792F905B0F0BD6D6265642D64657690
:109FF0002F746172676574732F68616C2F544152BE
:10A000004745545F53544D2F5441524745545F5375
:10A01000544D333246342F70696E6D61702E63007B
:10A0200070696E20213D202850696E4E616D652952
:10A030004E43000044AC000870B50C460546B0F134
:10A04000FF3F04D1A6220CA119A0FFF7CDFEC5F356
:10A05000031005F00F05FAF7A5FC022C88BF0024B9
:10A06000C268690003238B409A43C260C26804FA45
:10A0700001F11143C16070BD6D6265642D64657648
:10A080002F746172676574732F68616C2F5441522D
:10A090004745545F53544D2F5441524745545F53E5
:10A0A000544D333246342F70696E6D61702E6300EB
:10A0B00070696E20213D202850696E4E616D6529C2
:10A0C0004E430000884208BF7047B0F1FF3F04BF15
:10A0D0000846704710B5B1F1FF3F08BF10BD03A09F
:10A0E000FFF758FB4FF0FF3010BD000070696E6D38
:10A0F0006170206D69732D6D6174636800000000EC
:10A1000010B5B0F1FF3F08BF10BDB1F90020B2F1AA
:10A11000FF3F0DD0B1F90020824204D14C68B4F168
:10A12000FF3F0AD106E031F90C2FB2F1FF3FF1D128
:10A130004FF0FF3402A0FFF72DFB204610BD0000BA
:10A1400070696E6D6170206E6F7420666F756E64DD
:10A1500020666F72207065726970686572616C004C
:10A1600010B50446B0F1FF3F08BF10BDB1F90000C3
:10A17000B0F1FF3F13D000BFB1F90000A04209D1F8
:10A1800089682046FFF708FF2046BDE810400021FF
:10A19000FFF752BF31F90C0FB0F1FF3FECD1BDE832
:10A1A000104001A0FFF7F6BA636F756C64206E6F04
:10A1B000742070696E6F7574000000008160FFF795
:10A1C000AFBD00004168064800EB811210680168CD
:10A1D000C1F340110029FAD04068C0F3080070476D
:10A1E000380500202DE9F8430F46044616464B4932
:10A1F0003846FFF785FF054649493046FFF780FF9F
:10A2000001462846FFF75EFF2060B0F1FF3F04D112
:10A210006A2244A152A0FFF7E7FD20684FF0010831
:10A22000A0F18042B2F588424FF000051AD05349A0
:10A230005348B2F54C4F03D0B2F5504F27D038E019
:10A240000A6842F010020A600A6822F010020A60EE
:10A25000016841F010010160006800F010000090FA
:10A26000656026E04748016841F4003101600168FB
:10A2700021F4003101604448016841F4003101607B
:10A28000006800F400300090C4F8048011E00A680F
:10A2900042F020020A600A6822F020020A60016887
:10A2A00041F0200101600068052100F020000090CD
:10A2B00061601A493846FFF753FF19493046FFF7E6
:10A2C0004FFFB7F1FF3F03D001213846FFF7B4FE3F
:10A2D000B6F1FF3F03D001213046FFF7ADFE4FF44A
:10A2E0001651C4E902152561656125622783204660
:10A2F0006683FFF715FD2068A0F18041B1F5884124
:10A3000018BFBDE8F883214821464C22C0F80080E0
:10A31000BDE8F8431E48F6F753BC000090AA0008B9
:10A32000D8AA00086D6265642D6465762F74617229
:10A33000676574732F68616C2F5441524745545FB1
:10A3400053544D2F5441524745545F53544D33326B
:10A3500046342F73657269616C5F6170692E6300AA
:10A360006F626A5F732D3E7561727420213D2028F3
:10A37000554152544E616D65294E430024380240C8
:10A38000443802402038024040380240E0010020BA
:10A3900038070020034B59604068034941F82020EA
:10A3A00070470000E0010020180500202DE9F0436F
:10A3B00004464068DFF84C8183B008EB8019002721
:10A3C0000097D9F80000A66B3D46016811F0400FD8
:10A3D0001CBFC16811F0400F06D0E16911F0040FF5
:10A3E0001CBF01F004010091016811F0010F1CBFB6
:10A3F000416911F0010F05D0A18B009A01F40061B1
:10A4000011430091016811F0020F1CBF416911F066
:10A41000010F05D0A18B009A01F4806111430091D6
:10A42000016811F0080F1CBF406910F0010F05D042
:10A43000A08B009900F40070084300904846FAF79A
:10A44000A7F8009810F4006F01BF009810F4806F17
:10A45000009810F4007F51D1B9F82C0018B1B9F868
:10A460002E10411A2164B9F82E0050B9D4E90F0119
:10A47000401E814205D3A08B009900F480700843F0
:10A480000090A08B10F4005F18BF002E36D0226C15
:10A49000002A88BF94F8480030D9715D814229D1E3
:10A4A0002564A08B009900F4005008430090606878
:10A4B00008EB80100168CA6822F02002CA600168B7
:10A4C000CA6822F48072CA6001684A6922F00102F7
:10A4D0004A6102686FF020011160016849680191CA
:10A4E000C78590F83A10232914BF2021212180F834
:10A4F0003A1003E0691CCDB2AA42CED8009803B04E
:10A50000BDE8F083380500204268074800EB82135D
:10A5100018680268C2F3C012002AFAD0C1F308001A
:10A5200019684860704700003805002040680449F9
:10A5300001EB801000680068C0F340107047000015
:10A540003805002030B44FF0000C102906BF4FF43E
:10A5500000614160C0F804C0002A04BFC0F808C010
:10A56000C0F80CC00CD00121012A08BFC0E902C10B
:10A5700006D00224022A14BFC0E90241C0E9024CFD
:10A580004169B1F5007F07D0002B08BF4FF4802C44
:10A59000C0F814C003D000E00BB1002101E04FF47B
:10A5A0008271016130BCFFF783BB00002DE9F041EF
:10A5B000074600680024A0F560500E462546B0F11D
:10A5C000804018BFB0F5806F0CD0B0F5784F18BF41
:10A5D000B0F57C4F03D012A0FFF7DCF80BE0F9F7E1
:10A5E00023FD01E0F9F708FD044604E004EBD47014
:10A5F0004410681CC5B2B44201DD082DF6D3082D05
:10A6000006D80D4800EB450030F8020CB86102E0B6
:10A610000AA0FFF7BFF83846BDE8F041FFF748BB96
:10A6200053504920696E7374616E6365206E6F7458
:10A63000207365740000000078AC0008436F756CEF
:10A64000646E27742073657475702072657175650A
:10A650007374656420535049206672657175656E28
:10A66000637900002DE9F84F894604461F4690465D
:10A67000464948460A9EFFF743FD0090444940463C
:10A68000FFF73EFD824643493846FFF739FD8346D2
:10A6900041493046FFF734FD054651460098FFF723
:10A6A00011FD824629465846FFF70CFD01465046EB
:10A6B000FFF708FD2060B0F1FF3F04D1512237A120
:10A6C00045A0FFF791FB216849480025A1F1804290
:10A6D000B2F5983207D1016841F4805101600168F8
:10A6E00001F48051009122684249A2F18043B3F500
:10A6F000605307D10A6842F480420A600A6802F493
:10A70000804200922268A2F18043B3F5705307D1D2
:10A710000A6842F400420A60096801F400410091AD
:10A720002168A1F18042B2F59A3207D1016841F463
:10A7300000510160006800F4005000901349484641
:10A74000FFF70EFD12494046FFF70AFD1149384652
:10A75000FFF706FD6560A5603820E560A061A4F8FC
:10A760001C80A4F81E9027846684B6F1FF3F04BFC6
:10A770004FF40070606103D007493046FFF7F0FCEA
:10A780002046BDE8F84FFFF793BA000020AB000861
:10A7900068AB0008B0AB0008F8AB00086D626564F8
:10A7A0002D6465762F746172676574732F68616CB0
:10A7B0002F5441524745545F53544D2F54415247F3
:10A7C00045545F53544D333246342F7370695F6183
:10A7D00070692E63000000006F626A2D3E7370691D
:10A7E00020213D20285350494E616D65294E43007C
:10A7F00044380240403802400A4AD0F800C003689A
:10A8000013609B68C3F34003002BF8D089B2CCF8E7
:10A810000C10036801681160896811F0010FF9D00C
:10A82000D86870478407002010B504460068C068E7
:10A830008047606840680028206811D040688047E1
:10A8400061680246486803689A1A002A0CDC82682C
:10A850004A606168096800291CBF40688847E8E7CA
:10A860008068BDE8104000474868216800680969B1
:10A87000BDE81040084700684068004770B5164CB6
:10A880002068016911F0020F1CBFC16811F0020FAE
:10A8900004D06FF00201016100F048F820680169FE
:10A8A00011F0040F1ABFC16811F0040F70BD6FF0F2
:10A8B000040101612068456A084E3068281AB0F525
:10A8C0007A7F38BF70BDF8F72DFE216805F57A70E4
:10A8D0008863356070BD0000C8020020940100202C
:10A8E00002496FF00200096808617047FC07002008
:10A8F00003480068C16821F00201C1607047000090
:10A90000FC07002006480168002918BF7047012194
:10A9100001600549034808600020F8F725BE0000E3
:10A92000EC010020000C0040FC0700200148FFF76C
:10A930007BBF0000ACAC0008074810B5016839B90E
:10A94000012101600649054808600020F8F70CFE67
:10A950000448006810BD0000EC010020000C00401D
:10A96000FC070020240C0040034909684863C868BC
:10A9700040F00200C8607047FC07002070B54FF43B
:10A980007A7100FB01F5FFF7D7FF0446FFF7D4FF0C
:10A99000001BA842FAD370BD70B50546FFF7CCFF87
:10A9A0004FEA0004FFF7C8FF001BA842FAD370BDAE
:10A9B00010B500290AD00878002807D00548784447
:10A9C000F6F758F9002801D0002010BD024878445D
:10A9D00010BD0000F2150000EA15000010B50029B6
:10A9E0000AD00878002807D005487844F6F742F9DD
:10A9F000002801D0002010BD0248784410BD00009E
:10AA0000E2150000DA15000010B5044600680028C1
:10AA100006BF201D20602068211D884204D05622D8
:10AA200002490348FFF7E0F9206810BD74BF000831
:10AA300060BF00084A68096800EB620012F0010F6D
:10AA400001D002685158084730B4002804BF30BC18
:10AA5000704713684BB1526800EB620012F0010FAF
:10AA600001D00268D35830BC1847D2F804C01CF09B
:10AA7000010F18BFBCF1000FEDD130BC70474FF093
:10AA80004070E1EE100A7047F7F7C5B8F7F7FAB96A
:10AA90000200000000440040930300000900000091
:10AAA00000100140930300000B000000001401405F
:10AAB0001304000016000000001001409303000082
:10AAC000260000000014014013040000FFFF0000F6
:10AAD000FFFFFFFF000000000300000000440040F3
:10AAE000930300000A0000000010014093030000DF
:10AAF0000C000000001401401304000017000000C7
:10AB000000100140930300002700000000140140E2
:10AB100013040000FFFF0000FFFFFFFF0000000024
:10AB20000700000000300140930200001500000003
:10AB300000300140930200001F0000000038004078
:10AB40009302000023000000003800409302000040
:10AB50002C000000003C004013030000FFFF000039
:10AB6000FFFFFFFF00000000060000000030014072
:10AB70009302000014000000003001409302000026
:10AB80001E00000000380040930200002200000078
:10AB900000380040930200002B000000003C004001
:10ABA00013030000FFFF0000FFFFFFFF0000000095
:10ABB0000500000000300140930200001300000077
:10ABC00000300140930200001A00000000380040ED
:10ABD000930200001D0000000038004093020000B6
:10ABE0002A000000003C004013030000FFFF0000AB
:10ABF000FFFFFFFF000000000400000000300140E4
:10AC0000830200000F0000000030014083020000BA
:10AC10001900000000380040830200001C00000002
:10AC20000038004083020000FFFF0000FFFFFFFF2D
:10AC3000000000000000000000000000010203040A
:10AC400006070809000000000100000011000000D4
:10AC500002000000120000000300000000001110BC
:10AC6000000021100000311000001210000022101E
:10AC70000000321000000010000008001000180052
:10AC8000200028003000380000000000010203040A
:10AC9000010203040607080905A9000839A90008EC
:10ACA000F1A80008E1A8000869A9000898AC00080C
:10ACB000040200202F737464696E002F7374646F34
:10ACC0007574002F737464657272000089830008C4
:10ACD0000000000000000000000000001111111130
:10ACE00011111111102056657273696F6E3A203080
:10ACF0002E310000FF0000000200000000000000F4
:10AD0000FF0007000100000000000000FF0100003C
:10AD10000801000067000000FF02000010000000B2
:10AD200000000000FF040000080000000000000018
:10AD3000FF0500000800000000000000FF06000002
:10AD40000800000000000000FF07000008000000ED
:10AD500000000000FF0800000801000000000000E3
:10AD6000FF0900000800000000000000FF0A0000CA
:10AD70000800000000000000FF0B000008000000B9
:10AD800000000000FF0C00001001000000000000A7
:10AD9000FF0E00000801000000000000FF0F00008F
:10ADA0000801000000000000FF100000010000008A
:10ADB00000000000FF100100010000000000000082
:10ADC000FF1002000100000000000000FF1003005F
:10ADD0000100000000000000FF1100000100000061
:10ADE00001000000FF11010001000000010000004F
:10ADF000FF1200000100000000000000FF1201002F
:10AE00000100000000000000FF120200010000002D
:10AE100000000000FF12030001000000000000001D
:10AE2000FF1300000101000000000000FF130100FB
:10AE30000101000000000000FF14000001010000FB
:10AE400000000000FF1401000101000000000000EC
:10AE5000FF1402000101000000000000FF140300C5
:10AE60000101000000000000FF14040001010000C7
:10AE700000000000FF1500000101000000000000BC
:10AE8000FF1501000101000000000000FF15020095
:10AE90000101000000000000FF1503000101000097
:10AEA00000000000FF150400010100000000000088
:10AEB000FF1505000101000000000000FF1506005D
:10AEC0000101000000000000FF1507000101000063
:10AED00000000000FF16000001010000000000005B
:10AEE000FF1601000101000000000000FF16020033
:10AEF0000101000000000000FF1603000101000036
:10AF000000000000FF160400010100000000000026
:10AF1000FF1605000101000000000000FF160600FA
:10AF20000101000000000000FF1607000101000001
:10AF300000000000FF1700000101000000000000F9
:10AF4000FF1701000101000000000000FF170200D0
:10AF50000101000000000000FF17030001010000D4
:10AF600000000000FF1704000101000000000000C5
:10AF7000FF1705000101000000000000FF17060098
:10AF80000101000000000000FF17070001010000A0
:10AF900000000000FF180000010100000000000098
:10AFA000FF1801000101000000000000FF1802006E
:10AFB0000101000000000000FF1803000101000073
:10AFC00000000000FF180400010100000000000064
:10AFD000FF1805000101000000000000FF18060036
:10AFE0000101000000000000FF180700010100003F
:10AFF00000000000FF190000010100000000000037
:10B00000FF1901000101000000000000FF1902000B
:10B010000101000000000000FF1A00000101000013
:10B0200000000000FF1A0100010100000000000004
:10B03000FF1A02000101000000000000FF1A0300D7
:10B040000101000000000000FF1A040001010000DF
:10B0500000000000FF1A05000101000000000000D0
:10B06000FF1A06000101000000000000FF1A07009F
:10B070000101000000000000FF1B000004000000B0
:10B0800000000000FF1C00000400000000000000A1
:10B09000FF1D00000500000000000000FF1E000072
:10B0A0000501000000000000FF1F00000500000077
:10B0B00000000000FF200000080100000000000068
:10B0C000FF7D00000801000000000000FF7E00007E
:10B0D0000801000001000000FF7F000001000000E7
:10B0E000010000000021000001000000000000003D
:10B0F0000021010001000000010000000021020009
:10B100000100000000000000002103000100000019
:10B110000000000000210400010000000000000009
:10B1200000210500010000000000000000220000D6
:10B1300004000000070000000023000008000000D9
:10B14000F0000000002400010D00000080FEFFFF61
:10B15000002600010D00000080FFFFFF0028000115
:10B160000D00000080000000002A00010D0000001A
:10B1700080010000002C00010D00000080FEFFFF98
:10B18000002E00010D00000080FFFFFF00300001D5
:10B190000D00000080000000003200010D000000E2
:10B1A00080010000003400010D00000000000000DC
:10B1B000003600010D00000000000000004000000B
:10B1C0000100000000000000004001000400000039
:10B1D0000700000000410000070000000000000020
:10B1E00000420000070000000000000000430000D3
:10B1F00007000000000000000044000007000000FD
:10B2000000000000004500000700000000000000F2
:10B21000004600000700000000000000004700009A
:10B2200007000000000000000048000007000000C8
:10B2300000000000004900000100000000000000C4
:10B240000049010001000000010000000049020067
:10B25000010000000100000000490300010000009F
:10B26000010000000049040001000000010000008E
:10B27000004905000100000001000000004906002F
:10B280000100000001000000004A0000040000006E
:10B2900004000000004A0400040000000400000054
:10B2A000004B00000400000004000000004B0400FC
:10B2B0000400000004000000004C00000400000036
:10B2C00004000000004C0400040000000400000022
:10B2D000004D00000400000004000000004E0000CB
:10B2E0000400000004000000004E04000300000001
:10B2F00005000000005100000C00000000000000EC
:10B30000005300000C000000FC0F0000005500007E
:10B3100008000000070000000056000008000000C0
:10B3200000000000005700000801000000000000BD
:10B330000058000008010000000000000059000053
:10B3400001000000010000000059010001000000A0
:10B3500001000000005A0000010000000000000091
:10B36000005A01000300000000000000005B000024
:10B370000800000000000000005C00000800000061
:10B380001D000000005D0000060000000900000034
:10B39000005E00000200000002000000005E0200EB
:10B3A0000200000001000000005E04000200000036
:10B3B00000000000005F0000040000000100000029
:10B3C000005F0400040000000200000000600000B4
:10B3D000100000000A0000000062000001000000F0
:10B3E00001000000006201000100000001000000F7
:10B3F0000063000004000000080000000063040077
:10B4000002000000020000000064000007000000CD
:10B41000000000000065000008000000FF000000C0
:10B42000006600000100000001000000006700004D
:10B430000800000000000000006800000400000098
:10B44000080000000068040004000000070000007D
:10B450000069010001000000010000000069020015
:10B46000010000000100000000690300010000006D
:10B4700001000000006A000001000000010000005F
:10B48000006A01000100000001000000006A0200E3
:10B490000100000000000000006A0300010000003D
:10B4A00000000000006A040001010000000000002C
:10B4B000006A05000101000000000000006A0600AB
:10B4C0000100000000000000006A07000100000009
:10B4D00000000000006B00000800000001000000F8
:10B4E000006C00000800000020000000006D00005B
:10B4F0000800000064000000006E0000080000006A
:10B5000064000000006F000005000000070000005C
:10B510000070000005000000050000000071000040
:10B520000500000008000000007200000600000096
:10B530000000000000730000060000000000000092
:10B540000074000006000000000000000074060007
:10B55000010000000000000000750000060000006F
:10B5600000000000012100000100000000000000B8
:10B570000121010001000000000000000121020083
:10B580000100000000000000012200001000000087
:10B590000000000001240000040000000100000081
:10B5A0000124040004000000020000000125000046
:10B5B0000300000000000000012700010800000057
:10B5C0000000000001280001080000000000000049
:10B5D0000129000001000000000000000129010015
:10B5E0000400000000000000012905000100000027
:10B5F000000000000129060001000000000000001A
:10B60000012A00000200000000000000012A0200E0
:10B610000300000005000000012A050002000000F0
:10B6200000000000012A07000100000001000000E6
:10B63000012B00000100000000000000012B0100B0
:10B640000100000000000000012B020003000000C8
:10B6500000000000012C00000800000000000000B5
:10B66000012D00000100000001000000012E00007B
:10B670000400000001000000012E0400040000008E
:10B6800002000000012F0000100000000A0000006E
:10B690000131000001000000010000000131010043
:10B6A000010000000100000001320000080000005D
:10B6B0000A00000001330000030000000300000046
:10B6C00001340000080000001D00000001350000EA
:10B6D0000600000024000000013600000C000000FD
:10B6E000000000000138000002000000020000001D
:10B6F00001380200020000000100000001380400CF
:10B7000002000000000000000139000008000000F5
:10B7100000000000013A00000200000000000000EC
:10B72000013A02000100000000000000013A03009D
:10B730000100000001000000013B000004000000C7
:10B7400008000000013B04000200000003000000AC
:10B75000013B06000100000000000000013C000069
:10B760000400000007000000013C0400010000008C
:10B7700001000000013D000008000000FF00000083
:10B78000013E00000801000080000000013F0000B1
:10B790000300000000000000013F03000300000060
:10B7A00000000000013F0600010000000000000052
:10B7B000013F070001000000000000000140000000
:10B7C0000300000000000000014003000100000031
:10B7D0000000000001400400020000000000000022
:10B7E00001400600010000000000000001410000CF
:10B7F00005000000000000000141070001000000FA
:10B8000000000000014200001000000000000000E5
:10B81000014400002000000000000000014800007A
:10B820002000000000000000014C000008000000A3
:10B8300000000000014D00000100000001000000B8
:10B84000014D01000200000000000000014D030056
:10B850000100000001000000014D04000100000093
:10B8600000000000014D0500030000000000000082
:10B87000015000000800000000000000015100001D
:10B88000080000000000000001520000010000005C
:10B8900001000000015300000A0000000000000049
:10B8A0000221000008000000000000000222000049
:10B8B0000801000000000000022300000800000052
:10B8C0000000000002250000010000000000000050
:10B8D000022600000800000000000000022700000F
:10B8E000080100000000000002280000080000001D
:10B8F00000000000022A000001000000000000001B
:10B90000022B00000100000000000000022B0100DB
:10B910000100000000000000022B020001000000F6
:10B9200001000000022B03000100000000000000E5
:10B93000022B04000100000000000000022B0500A3
:10B940000100000000000000022B060001000000C2
:10B9500000000000022C00000200000000000000B7
:10B96000022D00000400000002000000022D04006F
:10B970000400000004000000022E0000040000008B
:10B9800002000000022E0400040000000400000079
:10B99000022F00000500000000000000022F05003B
:10B9A0000100000000000000022F0600010000005E
:10B9B00000000000022F070001000000000000004E
:10B9C0000230000010000000000000000233000000
:10B9D000080100000000000002340000080100001F
:10B9E0000000000002360000080100000000000016
:10B9F00002380000080100000000000002390000C9
:10BA00000801000000000000023A000008010000E8
:10BA100000000000023B00000801000000000000E0
:10BA2000023C00000801000000000000023D000090
:10BA30000801000000000000023E000008010000B4
:10BA400000000000023F00000801000000000000AC
:10BA50000240000008010000000000000241000058
:10BA60000801000000000000024200001001000078
:10BA7000000000000244000010010000000000006F
:10BA8000024600002001000000000000024A000001
:10BA90000401000000000000024A0400040100004C
:10BAA00000000000024B0000040100000000000044
:10BAB000024B04000401000000000000024C0000E2
:10BAC0000401000000000000024C0400040100001A
:10BAD00000000000024D0000040100000000000012
:10BAE000024D04000401000000000000024E0000AE
:10BAF0000401000000000000024F000003010000EC
:10BB000000000000024F03000301000000000000DD
:10BB10000250000008000000000000000251000078
:10BB200008000000000000000252000001000000B8
:10BB300000000000025201000100000000000000AF
:10BB40000252020001000000000000000253000049
:10BB5000010000000000000002540000010000008D
:10BB6000000000000254010001000000000000007D
:10BB70000254020002000000000000000254040011
:10BB80000300000000000000025407000101000053
:10BB90000000000002550000080000000000000046
:10BBA00002560000080000000000000002570000DC
:10BBB0000801000000000000025800000801000019
:10BBC0000000000002590000010000000000000019
:10BBD000025901000100000001000000025A0001AA
:10BBE0000800000000000000025B020106000000E7
:10BBF00000000000025C00011000000000000000D6
:10BC0000025E00000401000000000000025F00006E
:10BC100005010000000000000260000005010000B6
:10BC200000000000026100000501000000000000AB
:10BC30000121000008000000000000002D8F000816
:10BC40000000000030313233343536373839414264
:10BC5000434445464030580030313233343536376E
:10BC6000383961626364656640307800040000081A
:10BC700000000000000000020001000010000000B1
:10BC80000000000000000000303132333435363718
:10BC900038396162636465667870003031323334FC
:10BCA0003536373839414243444546585000000044
:10BCB00002400000000000A000000000054000005D
:10BCC000000000C8000000000C4000000000409C84
:10BCD00000000000194000000020BCBE0000000071
:10BCE00034400000BFC91B8E00000004B5400000B6
:10BCF000504BCFD06607E2CF010000006C4100003E
:10BD00003E8251AADFEEA73401000000D9420000B4
:10BD1000DCB5A0E23A301F97FFFFFFFFB4450000FB
:10BD2000FD25A0C8E9A3C14FFFFFFFFFFF3F0000B3
:10BD30000000008000000000FF3F000000000080C5
:10BD4000000000000000000000000000018E00085C
:10BD500000000000000000005F8800086188000803
:10BD600000000000000000000000000000000000D3
:10BD700000000000000000000000000048FFFFFF7E
:10BD800000000000258900081D890008E1880008DE
:10BD90006189000821890008000000008D880008E2
:10BDA0000000000000000000519100085F910008B1
:10BDB000599100085391000844FFFFFF0000000064
:10BDC00000000000000000002CFFFFFF000000004A
:10BDD000619100086B910008CD91000800000000FF
:10BDE00000000000BD920008BD920008BD9200084E
:10BDF000BD920008BD920008BD92000809830008AA
:10BE000000000000000000005B8300085D83000864
:10BE10000000000000000000ED830008EF83000830
:10BE20000000000000000000000000000000000012
:10BE30006D85000800000000000000000000000008
:10BE4000B98500088D85000869860008000000009B
:10BE50000000000000000000000000005F880008F3
:10BE600061880008000000000000000000000000E1
:10BE70000000000048FFFFFF0000000025890008C7
:10BE80001D890008E18800086189000821890008EF
:10BE9000000000008D880008000000000000000085
:10BEA000519100085F9100085991000853910008D2
:10BEB00044FFFFFF00000000000000000000000041
:10BEC0000000000000000000258900081D8900080E
:10BED000E18800086189000821890008000000004D
:10BEE0008D88000800000000000000005B8300084F
:10BEF0005D830008BD920008BD920008FCFFFFFFB3
:10BF00000000000000000000000000000000000031
:10BF10000000000000000000000000000000000021
:10BF200000000000BD920008BD920008BD9200080C
:10BF3000BD920008BD920008BD9200080983000868
:10BF400000000000000000005B8300085D83000823
:10BF5000FCFFFFFF000000000000000000000000E8
:10BF60005F707472203D3D202854202A29265F648A
:10BF7000617461006D6265642D6465762F6170691E
:10BF80002F53696E676C65746F6E5074722E680003
:10BF9000E4C000089401002034010000D001000832
:10BFA00018C10008C8020020402800002C02000828
:10BFB0001C00000043000000F8FFFFFF0C00000021
:10BFC0000E0000000F0000002E0000001001000015
:10BFD00043000000F8FFFFFF004040404040404069
:10BFE000404041414141414040404040404040404C
:10BFF00040404040404040404005020202020202F0
:10C00000020202020202020202202020202020203E
:10C010002020200202020202020290909090909052
:10C020001010101010101010101010101010101010
:10C030001010101002020202020288888888888884
:10C040000808080808080808080808080808080870
:10C050000808080802020202400000000000000078
:10C0600000000000000000000000000000000000D0
:10C0700000000000000000000000000000000000C0
:10C0800000000000000000000000000000000000B0
:10C0900000000000000000000000000000000000A0
:10C0A0000000000000000000000000000000000090
:10C0B0000000000000000000000000000000000080
:10C0C0000000000000000000000000000000000070
:10C0D000000000000000000000000000E9D1FFFFA8
:10C0E000F5D1FFFF51041CBD0105320132023203BC
:10C0F0000A150414091B41012B295881AA030D318B
:10C10000041EC194C11502030A0E054603030E1B4B
:08C1100029E01AFF01011000F3
:040000050800019559
:00000001FF
